:100000000C946C040C9496040C9496040C94960432
:100010000C9496040C9496040C9496040C949604F8
:100020000C9496040C9496040C9496040C949604E8
:100030000C9496040C9496040C9496040C94B0467C
:100040000C9496040C9496040C94D6440C94960448
:100050000C944A450C9420450C9496040C949604F8
:100060000C9496040C9496040C9480450C9496047D
:100070000C9496040C9496040C9496040C94960498
:100080000C9496040C9496040C94960400002000A2
:100090002300260029003EBD3CBEBEBD3CBDBC21A8
:1000A000BD002044697228732900202020202020D0
:1000B000202000206279746573002046696C6528F1
:1000C0007329202020002020202020202020002014
:1000D000003C4449523E00200020566F6C756D650F
:1000E00020696E2064726976652043206861732000
:1000F0006E6F206C6162656C0020004F5554204F7C
:10010000462044415441004F5554204F462044411D
:100110005441002D2D2D2D2D2D2D2D2D2D2D2D2D01
:100120002D2D2D2D2D2D2D2D2D2D2D2D2D2D2D2DFF
:100130002D2D2D2D2D2D2D0049324320454550527A
:100140004F4D20284229002D2D2D2D2D2D2D2D2DCB
:100150002D2D2D2D2D2D2D2D2D2D2D2D2D2D2D2DCF
:100160002D2D2D2D2D2D2D2D2D2D2D00494E542095
:10017000454550524F4D20284529002D2D2D2D2D20
:100180002D2D2D2D2D2D2D2D2D2D2D2D2D2D2D2D9F
:100190002D2D2D2D2D2D2D2D2D2D2D2D2D2D2D00BC
:1001A0004D454D4F5259204D4150002D2D2D2D2D97
:1001B0002D2D2D2D2D2D2D2D2D2D2D2D2D2D2D2D6F
:1001C0002D2D2D2D2D2D2D2D2D2D2D2D2D2D2D008C
:1001D0005352414D20494E464F524D4154494F4E86
:1001E00000504545CB4142D34144C34449CE524ED1
:1001F000C45351D2434852A441D200535445D00075
:1002000054CF004E6F742061206469726563746F0F
:100210007279004469726563746F7279206E6F74CD
:1002200020666F756E6400534156494E472E2E2E40
:100230000053442066696C65206572726F722E00EF
:100240004C4F4144494E472E2E2E00444F4E450000
:10025000444F4E45004C4953D44E45D75255CE4E8F
:100260004558D44C45D449C6474F54CF474F5355B2
:10027000C25245545552CE5245CD464FD2494E50AA
:1002800055D45052494ED442524541CB455849D499
:100290004D45CD4545D05241CD504F4BC5444154BD
:1002A000C1524541C4524553544F52C5BFA7414F57
:1002B00055D44F55D4574149D4454EC45253454562
:1002C000C4434CD3504C4FD44C494EC5524543D4F3
:1002D000434952434CC5434841D24745545049D8FD
:1002E0004C4F434154C54C494D49D4454C4953D4D6
:1002F000454C4F41C445464F524D41D4455341565C
:10030000C545504F4BC545504545CB4544554DD04F
:100310004449D24C4F41C4534156C54445CC4DC4C9
:1003200052C443C443484B4453CB424C4953D44238
:100330004C4F41C442464F524D41D442534156C5A1
:1003400042504F4BC542504545CB4244554DD04994
:100350004E4B45D9504C41D953544FD04745D4000A
:10036000627265616B21003F4E6F7420656E6F7520
:100370006768206D656D6F727921003F53796E74E7
:100380006178204572726F72003F496E76616C69C8
:1003900064206C696E65206E756D626572003F4900
:1003A0006E76616C69642065787072657373696FCD
:1003B0006E000820080052454144592E00000000FC
:1003C00000000102000000000000095E00000000C3
:1003D00000007131000000797361773200006378AA
:1003E00064653433000020766674723500006E62F6
:1003F00068677A360000006D6A75373800002C6B2C
:10040000696F303900002E2D6C85708300000081EB
:10041000008727000000000D2B00230000003C0097
:100420000000007F000031003437000000302E3221
:100430003536381B00002B332D2A39000000000010
:100440000000000000000102000000000000098917
:1004500000000000000051210000005953415722C4
:100460000000435844452488000020564654522535
:1004700000004E4248475A260000004D4A552F289A
:1004800000003B4B494F3D2900003A5F4C84503FF0
:1004900000000082008660000000000D2A00270096
:1004A00000003E000000007F0000310034370000F3
:1004B00000302E323536381B00002B332D2A390000
:1004C00000000000007C3C3E5E2B3D3F2F5B5D3B0F
:1004D0002C2A225C0054696E792042415349432002
:1004E000286329203230323620442E204B72697323
:1004F00074656E2076322E30202020000608200001
:10050000000000000000004040404040004000501B
:1005100050500000000000000050F850F85000203B
:1005200070A0702870200000C8D0205898000020CB
:10053000508040A89068004040400000000000103B
:1005400020404040201000402010101020400000AB
:1005500020A870A8200000002020F8202000000023
:1005600000000000101000000000F8000000000073
:100570000000000010000000081020408000007003
:1005800088A8A888700000206020202070000070DB
:1005900088102040F80000F81020108870000090AB
:1005A0009090F810100000F880F00888700000703B
:1005B00080F08888700000F80810204080000070EB
:1005C0008870888870000070888878087000000043
:1005D000002000002000000000200020204000003B
:1005E00018608060180000000078007800000000AB
:1005F000C0300830C0000060902020002000007053
:100600008898A890887000205088F888880000F0AA
:1006100088F08888F000007088808088700000F082
:1006200088888888F00000F880F88080F80000F85A
:1006300080F080808000007088809888700000883A
:1006400088F88888880000702020202070000038FA
:10065000101010906000008890E0A090880000804A
:1006600080808080F8000088D8A8A888880000884A
:1006700088C8A8988800007088888888700000F072
:1006800088F08080800000708888A890680000F062
:1006900088F0A0908800007880700808F00000F8CA
:1006A000202020202000008888888888700000880A
:1006B000888888502000008888A8A8A85000008852
:1006C000502050888800008888502020200000F8A2
:1006D00008102040F80000E080808080E0000000EA
:1006E0008040201008000038080808083800002062
:1006F00050000000000000000000000000F8008032
:100700004000000000000000601070906000008059
:1007100080E09090E0000000007080807000001089
:1007200010709090700000006090F08070000030B9
:1007300040E0404040000000609070101060008079
:1007400080E0909090000020002020207000001099
:10075000003010101060008090A0C0A090000060D9
:1007600020202020700000000050A8A8A800000051
:1007700000F0888888000000006090906000000011
:10078000006090F080800000006090F01010000089
:1007900000B04840400000003040201060000040A1
:1007A00040E0404040000000009090906000000059
:1007B00000888850200000000088A8A85000000091
:1007C0008850205088000000009090604080000019
:1007D00000F02040F00000204040804040200020F9
:1007E0002020202020200020101008101020004081
:1007F000A81000000000000000000000000000F849
:10080000F8F8F8F8F8F8009060107090600000A810
:100810005088F888880000007088F0C8B080008890
:100820007088888870000090006090906000008858
:1008300000888888700000900090909060000070A0
:100840008060906010E00040A040000000000000C8
:1008500000F8C0C0C0C0C00000F818181818180070
:10086000002100240027002A000000220025002883
:10087000002B000202020202020202040404040429
:10088000040404030303030303030301010101013F
:100890000101010102040810204080010204081037
:1008A000204080010204081020408001020408104A
:1008B0002040800000000203000A0B000000000539
:1008C0000409080000000000000000000000000013
:1008D000000000250000E04611241FBECFEFD0E449
:1008E000DEBFCDBF14E0A0E0B1E0E2E5F2EA00E057
:1008F0000BBF02C007900D92A831B107D9F723E2D0
:10090000A8E1B4E001C01D92AC39B207E1F714E0F0
:10091000CCE6D4E004C02197FE010E94A150CB3662
:10092000D107C9F70E9443470C9427510C9400004B
:100930008091722090917E20E0917320F09174203C
:1009400031962491492F421B550B84171506CCF084
:10095000E491A0918420B091852080917F209D0119
:10096000E89F200D311D1124F9019D01989F200D54
:10097000311D11242E173F0740F080818D93119275
:10098000F9CFE491E80FE093722008952F923F92FF
:100990004F925F926F927F928F929F92AF92BF928F
:1009A000CF92DF92EF92FF920F931F93CF93DF933B
:1009B00000D000D000D0CDB7DEB7009173201091E9
:1009C0007420F8013296549198012F5F3F4FF9013E
:1009D000F490F8019491F9012491451B429FA001E4
:1009E0001124DA011396282F277078E0721B9111D9
:1009F00005C0F801EA0FFB1F94911196F11005C094
:100A0000F801EA0FFB1FF4901196F92FF770F983A4
:100A1000E92FE695E695E695FF2309F498C0EF5F88
:100A200090917F20822E912C4981480D592D511D86
:100A30005E834D832FEF30E069010D8002C0D594B5
:100A4000C7940A94E2F7472F50E05A83498301C0C4
:100A5000220F7A95EAF7AC2CE13009F0A12CA22AFA
:100A60004D815E81485051092FEF30E002C035952D
:100A700027954A95E2F7E22E292E312C8695869508
:100A80008695969FB0011124860F972F911DB12C4A
:100A90002E2F2150330B3C832B83FB1409F481C090
:100AA000E0916F20F0917020E80FF91FD0802D2D7C
:100AB0002A212083BD016F5F7F4FF801EA0FFB1FE2
:100AC0002491E0916F20F0917020E80FF91F422FE0
:100AD00050E0082C02C0559547950A94E2F7308102
:100AE000432B40834B805C80460E571E3C016A1AA4
:100AF0007B0AD301A60FB71F40916F205091702041
:100B000030E0098002C0220F331F0A94E2F7641517
:100B1000750500F5FA01EA0FFB1FD0802083F8016C
:100B2000E60FF71F249140916F2050917020A40F81
:100B3000B51F422F50E0082C02C0559547950A94E6
:100B4000E2F73C91432B4C936F5F7F4FD2CF38E05D
:100B5000398366CFED81FE813897B0F4FD0131977E
:100B6000E40FF51FDC204081D42AD08240916F2011
:100B700050917020A40FB51FEC912E2B2C93B394A1
:100B8000820D931DDB0189CFFA01EA0FFB1FD08094
:100B90004D815E814830510549F34D2D4E214083F2
:100BA000E5CF26960FB6F894DEBF0FBECDBFDF911E
:100BB000CF911F910F91FF90EF90DF90CF90BF905A
:100BC000AF909F908F907F906F905F904F903F90ED
:100BD0002F900895CF938A30B9F180F5882391F151
:100BE0008830B9F1C82F80917120E0917320F09185
:100BF0007420E49120917F2098E0299F9001112496
:100C00002E1B31094C2F60917220821713064CF075
:100C1000109271200E9498044C2F60917220809154
:100C200071200E94C604E0917320F0917420849199
:100C3000E0917120E80FE093712004C08D30C9F07D
:100C40008E3081F6CF91089510927120CF910C943F
:100C50009804E0917320F0917420E49180917120C8
:100C60008E1B8093712040E260917220CF910C9492
:100C7000C60410927120E6CFCF93DF93EC018991E7
:100C8000882319F00E94EA05FACFDF91CF910895E9
:100C9000CF93DF93FC018281938190938023809393
:100CA0007F2384819581A681B7818093812390934E
:100CB0008223A0938323B093842380859185A2858A
:100CC000B3858093852390938623A0938723B09345
:100CD0008823DF011C96CF014996C9E8D3E22D9104
:100CE0002993A817B907D9F7818D928D90939723EF
:100CF000809396238DE793E2DF91CF910895282F7B
:100D000090916E2081E0913208F042C080914A209B
:100D10008111FCCF80916D2032E030934A202093E6
:100D200049202FEF209348202DE430E230934720D4
:100D30002093462010924520909344201092432007
:100D400090914320880F892B8093432080914220EB
:100D5000813029F510924220809143208093BB007E
:100D60008091BC0083FDF8CF85EC8093BC0080911E
:100D70004A208230E1F3809148208F3F91F08091AA
:100D80004820803281F080914820803371F084E0E7
:100D900010924C2010926E2010924B20089585EEF8
:100DA000E4CF80E0F5CF82E0F3CF83E0F1CF109283
:100DB000712010927220E0918420F0918520909112
:100DC0007F2080917E209F01989F200D311D11244E
:100DD000C901E817F90711F01192FBCF089580912E
:100DE0007C2090917D2086309140F9F460917720AD
:100DF000709178208091792090917A200E94234FE1
:100E000023E333E34EE752E40E94B14F20E030E0A9
:100E100043E853E40E94B14F20E030E04AE754E455
:100E20000E947B4E0E94F44E0895209177203091CD
:100E300078204091792050917A20A0E0BEE40E9471
:100E4000374E28EE33E040E050E00E944A4ECA019F
:100E5000B90108954F925F926F927F928F929F9205
:100E6000AF92BF92CF92DF92EF92FF92CF93DF9338
:100E700000D000D0CDB7DEB74C012A013B01109263
:100E8000B0001092B100892B09F042C0579A0E941D
:100E9000EF06460E571E681E791E21EE3CEA3A8385
:100EA00029830E94EF066415750586059705E0F411
:100EB00089819A819695879529813A812170332776
:100EC0003195219531092227347B282739273A8308
:100ED000298320FF07C05F9A89818770815008F3BA
:100EE0000000FCCF5F98F8CF5F980F900F900F90A5
:100EF0000F90DF91CF91FF90EF90DF90CF90BF9058
:100F0000AF909F908F907F906F905F904F900895DB
:100F10009091B00092609093B0009091B100916078
:100F20009093B100579AB12CA12C60E072E18AE74E
:100F300090E0A50194010E94184E29833A834B83C7
:100F40005C8369017A0131E0C31AD108E108F10834
:100F50008FEFC816D104E104F10409F054F581E0E3
:100F60008093B100411451046104710409F4AAC0D2
:100F7000ACE3B0E0A30192010E94374E28EE33E0CB
:100F800040E050E00E944A4E20933E2030933F20A4
:100F90004093402050934120C092B3008091B00014
:100FA0008F778093B0008091B00080648093B00010
:100FB0009CCF60E472E48FE090E0A50194010E9470
:100FC000184E69017A0191E0C91AD108E108F108C7
:100FD00082E02FEFC216D104E104F10409F204F219
:100FE00060E970ED83E090E0A50194010E94184E45
:100FF00069017A0181E0C81AD108E108F10883E0AB
:101000009FEFC916D104E104F10409F00CF4A8CF54
:1010100068E478EE81E090E0A50194010E94184E0A
:1010200069017A0181E0C81AD108E108F10884E079
:101030009FEFC916D104E104F10409F00CF490CF3C
:1010400064E274EF80E090E0A50194010E94184EE4
:1010500069017A0181E0C81AD108E108F10885E048
:101060009FEFC916D104E104F10409F008F478CF28
:1010700062E17AE780E090E0A50194010E94184EB9
:1010800069017A0181E0C81AD108E108F10886E017
:101090009FEFC916D104E104F10409F008F460CF10
:1010A000C980DA80EB80FC808AE0F594E794D794DD
:1010B000C7948A95D1F721E0C21AD108E108F10856
:1010C00087E04ECF8FEF9FEFDC0180933E2090931F
:1010D0003F20A0934020B09341205ECFCF93DF9379
:1010E0009EE19093712080937220C3EDD8E0FE01C1
:1010F0008491882321F021960E94EA05F8CFDF91A0
:10110000CF91089582508A3088F5E82FF0E0E557B6
:10111000F74F0C94A150B308B70895089B08B60880
:10112000B6089F08A508A908AF08809180008F77AE
:10113000809380000895809180008F7DF9CF809109
:10114000B0008F778093B00008958091B0008F7DBC
:10115000F9CF809190008F778093900008958091CF
:1011600090008F7DF9CF84B58F7784BD089584B5C5
:101170008F7DFBCF1F93CF93DF93282F30E0F901B2
:10118000ED54F74F8491F901ED56F74FD491F901E1
:10119000ED58F74FC491CC23A9F0162F81110E946E
:1011A0008208EC2FF0E0EE0FFF1FE759F74FA591F3
:1011B000B4918FB7F894EC91111108C0D095DE234B
:1011C000DC938FBFDF91CF911F910895DE2BF8CF75
:1011D000CF93DF9390E0FC01ED56F74F24918D58AB
:1011E000974FFC0184918823D1F090E0880F991FDC
:1011F000FC01E15AF74FA591B491FC01E759F74F73
:10120000C591D49161110EC09FB7F8948C91E22FD3
:10121000E0958E238C932881E223E8839FBFDF91A2
:10122000CF9108958FB7F894EC91E22BEC938FBF98
:10123000F6CF3FB7F89480913A2090913B20A0914F
:101240003C20B0913D2026B5A89B05C02F3F19F04A
:101250000196A11DB11D3FBFBA2FA92F982F882736
:10126000BC01CD01620F711D811D911D42E0660F11
:10127000771F881F991F4A95D1F708958F929F92E3
:10128000AF92BF92CF92DF92EF92FF926B017C01FF
:101290000E9419094B015C01C114D104E104F1045D
:1012A000B9F00E941909681979098A099B09683EF1
:1012B00073408105910580F321E0C21AD108E1084D
:1012C000F10888EE880E83E0981EA11CB11CE4CFC3
:1012D000FF90EF90DF90CF90BF90AF909F908F9056
:1012E00008952FB7F894609136207091372080913F
:1012F0003820909139202FBF0895089508950F93B5
:10130000CF93DF93E5E7F0E2A785B089C091B11FE5
:10131000D091B21F8285AC0FBD1F02B10F7703C001
:1013200000FA07F902B90D90000007FA07F902B9AF
:1013300000000000000006FA07F902B900000000F2
:10134000000005FA07F902B900000000000004FAE5
:1013500007F902B900000000000003FA07F902B91A
:1013600000000000000002FA07F902B900000000C6
:10137000000001FA07F902B98A9591F60000000011
:1013800000FA07F902B902B10F7707FB07F902B9B2
:10139000DF91CF910F9108950F93CF93DF93E5E7FE
:1013A000F0E2A785B089C091B11FD091B21F8285AC
:1013B000AC0FBD1F02B10F7703C000FA07F902B9E5
:1013C0000D9007FA07F902B90000000006FA07F9C4
:1013D00002B90000000005FA07F902B90000000098
:1013E00004FA07F902B90000000003FA07F902B98C
:1013F0000000000002FA07F902B900008A9501FA1C
:1014000007F902B9D1F6000000FA07F902B902B1F2
:101410000F7707FB07F902B9DF91CF910F9108957C
:101420000F93CF93DF93E5E7F0E2A785B089C091F2
:10143000B11FD091B21F8285AC0FBD1F02C0000C3E
:1014400002B80D90000002B800000000000C02B8C5
:1014500000000000000C02B800000000000C02B800
:1014600000000000000C02B800000000000C02B8F0
:101470000000000C8A9502B811F70000000C02B8B9
:101480000000000000001798DF91CF910F910895A0
:101490000F93CF93DF93E5E7F0E2A785B089C09182
:1014A000B11FD091B21F8285AC0FBD1F8E3191F05C
:1014B0008D3151F08C3149F08B3141F08A3139F066
:1014C000893131F0883129F01CC032C048C05EC07B
:1014D00074C08AC00D9002B80000000C02B8000071
:1014E000000C02B80000000C02B80000000C02B8AA
:1014F0000000000C02B80000000C02B80000000C54
:1015000002B80D9002B80000000C02B80000000CF8
:1015100002B80000000C02B80000000C02B8000085
:10152000000C02B80000000C02B80000000C02B869
:101530000D9002B80000000C02B80000000C02B8C8
:101540000000000C02B80000000C02B80000000C03
:1015500002B80000000C02B80000000C02B80D90A8
:1015600002B80000000C02B80000000C02B8000035
:10157000000C02B80000000C02B80000000C02B819
:101580000000000C02B80000000C02B80D9002B878
:101590000000000C02B80000000C02B80000000CB3
:1015A00002B80000000C02B80000000C02B80000F5
:1015B000000C02B80000000C02B80D9002B8000048
:1015C000000C02B80000000C02B80000000C02B8C9
:1015D0000000000C02B80000000C02B80000000C73
:1015E00002B80000000C02B80D9002B80000000C18
:1015F00002B80000000C02B80000000C02B80000A5
:10160000000C02B80000000C02B80000000C02B888
:101610000000000C02B80D9002B80000000C02B8E7
:101620000000000C02B80000000C02B80000000C22
:1016300002B80000000C02B80000000C02B8000064
:10164000000C02B80D9002B80000000C02B80000B7
:10165000000C02B80000000C02B80000000C02B838
:101660000000000C02B80000000C02B80000000CE2
:1016700002B80D9002B80000000C02B80000000C87
:1016800002B80000000C02B80000000C02B8000014
:10169000000C02B80000000C02B80000000C02B8F8
:1016A0000D9002B80000000C02B80000000C02B857
:1016B0000000000C02B80000000C02B80000000C92
:1016C00002B80000000C02B80000000C02B80D9037
:1016D00002B80000000C02B80000000C02B80000C4
:1016E000000C02B80000000C02B80000000C02B8A8
:1016F0000000000C02B80000000C02B80D9002B807
:101700000000000C02B80000000C02B80000000C41
:1017100002B80000000C02B80000000C02B8000083
:10172000000C02B80000000C02B80D9002B80000D6
:10173000000C02B80000000C02B80000000C02B857
:101740000000000C02B80000000C02B80000000C01
:1017500002B80000000C02B80D9002B80000000CA6
:1017600002B80000000C02B80000000C02B8000033
:10177000000C02B80000000C02B80000000C02B817
:101780000000000C02B80D9002B80000000C02B876
:101790000000000C02B80000000C02B80000000CB1
:1017A00002B80000000C02B80000000C02B80000F3
:1017B000000C02B80D9002B80000000C02B8000046
:1017C000000C02B80000000C02B80000000C02B8C7
:1017D0000000000C02B80000000C02B80000000C71
:1017E00002B80D9002B80000000C02B80000000C16
:1017F00002B80000000C02B80000000C02B80000A3
:10180000000C02B80000000C02B80000000C02B886
:101810000D9002B80000000C02B80000000C02B8E5
:101820000000000C02B80000000C02B80000000C20
:1018300002B80000000C02B80000000C02B80D90C5
:1018400002B80000000C02B80000000C02B8000052
:10185000000C02B80000000C02B80000000C02B836
:101860000000000C02B80000000C02B80D9002B895
:101870000000000C02B80000000C02B80000000CD0
:1018800002B80000000C02B80000000C02B8000012
:10189000000C02B80000000C02B80D9002B8000065
:1018A000000C02B80000000C02B80000000C02B8E6
:1018B0000000000C02B80000000C02B80000000C90
:1018C00002B80000000C02B80D9002B80000000C35
:1018D00002B80000000C02B80000000C02B80000C2
:1018E000000C02B80000000C02B80000000C02B8A6
:1018F0000000000C02B80D9002B80000000C02B805
:101900000000000C02B80000000C02B80000000C3F
:1019100002B80000000C02B80000000C02B8000081
:10192000000C02B80D9002B80000000C02B80000D4
:10193000000C02B80000000C02B80000000C02B855
:101940000000000C02B80000000C02B80000000CFF
:1019500002B80D9002B80000000C02B80000000CA4
:1019600002B80000000C02B80000000C02B8000031
:10197000000C02B80000000C02B80000000C02B815
:101980000D9002B80000000C02B80000000C02B874
:101990000000000C02B80000000C02B80000000CAF
:1019A00002B80000000C02B80000000C02B80D9054
:1019B00002B80000000C02B80000000C02B80000E1
:1019C000000C02B80000000C02B80000000C02B8C5
:1019D0000000000C02B80000000C02B80D9002B824
:1019E0000000000C02B80000000C02B80000000C5F
:1019F00002B80000000C02B80000000C02B80000A1
:101A0000000C02B80000000C02B80D9002B80000F3
:101A1000000C02B80000000C02B80000000C02B874
:101A20000000000C02B80000000C02B80000000C1E
:101A300002B80000000C02B8000000001798DF9107
:101A4000CF910F910895209175203091762080914B
:101A50007C2090917D20281739070CF457C08CEA20
:101A600093E09093890080938800109276201092E2
:101A700075208091772090917820A0917920B09165
:101A80007A200196A11DB11D809377209093782034
:101A9000A0937920B0937A2080913E2090913F20AE
:101AA000A0914020B0914120892B8A2B8B2B51F1A2
:101AB00080913E2090913F20A0914020B091412004
:101AC000181619061A061B069CF480913E20909168
:101AD0003F20A0914020B09141200197A109B10978
:101AE00080933E2090933F20A0934020B0934120CC
:101AF0008091752090917620019690937620809326
:101B0000752008951092B1002F98F2CF2091752082
:101B10003091762080918320082E000C990B281795
:101B2000390731F78AE490E0909389008093880028
:101B30008EE89BE190931E2080931D20D9CFAF9219
:101B4000BF92CF92DF92EF92FF920F931F93CF93AA
:101B5000DF936C017B018B01040F151FEB015E010C
:101B6000AE18BF08C017D10759F06991D601ED91A1
:101B7000FC910190F081E02DC6010995892B79F740
:101B8000C501DF91CF911F910F91FF90EF90DF90F2
:101B9000CF90BF90AF900895FC01538D448D252FB9
:101BA00030E0842F90E0821B930B541710F0CF96F7
:101BB000089501970895FC01918D828D981761F029
:101BC000A28DAE0FBF2FB11D5D968C91928D9F5F40
:101BD0009F73928F90E008958FEF9FEF0895FC011F
:101BE000918D828D981731F0828DE80FF11D858DD2
:101BF00090E008958FEF9FEF0895FC01918D228D65
:101C0000892F90E0805C9F4F821B91098F739927E9
:101C1000089589E892E20E94FD0D21E0892B09F4E4
:101C200020E0822F0895FC01A48DA80FB92FB11DCB
:101C3000A35ABF4F2C91848D90E001968F73992702
:101C4000848FA689B7892C93A089B1898C918370E0
:101C500080648C93938D848D981306C00288F389D9
:101C6000E02D80818F7D80830895EF92FF920F9306
:101C70001F93CF93DF93EC0181E0888F9B8D8C8D38
:101C800098131AC0E889F989808185FF15C09FB72C
:101C9000F894EE89FF896083E889F98980818370EF
:101CA000806480839FBF81E090E0DF91CF911F919E
:101CB0000F91FF90EF900895F62E0B8D10E00F5FBF
:101CC0001F4F0F731127E02E8C8D8E110CC00FB695
:101CD00007FCFACFE889F989808185FFF5CFCE012D
:101CE0000E94130EF1CFEB8DEC0FFD2FF11DE35A87
:101CF000FF4FF0829FB7F8940B8FEA89FB898081B0
:101D00008062CFCFCF93DF93EC01888D8823B9F029
:101D1000AA89BB89E889F9898C9185FD03C08081F6
:101D200086FD0DC00FB607FCF7CF8C9185FFF2CF73
:101D3000808185FFEDCFCE010E94130EE9CFDF91A8
:101D4000CF91089580E090E0892B29F00E94090E40
:101D500081110E94000080E090E0892B49F080E032
:101D600090E0892B29F00E94000081110C94000062
:101D7000089585ED8093BC008091BC0084FDFCCF6C
:101D800010924A2008952091FA1F260F3327331FFF
:101D900021323105ECF420914A20FC0190E080E0F2
:101DA000243069F082E00895A091FA1F2191AC01DE
:101DB0004652504EA40FB52FB11D2C930196861795
:101DC00098F38091FA1F680F6093FA1F80E00895DE
:101DD00081E008950895E091262080912520E8175C
:101DE00030F4F0E0E654F04E808190E008958FEFFB
:101DF0009FEF089590912620809125202FEF3FEFAF
:101E0000981748F4E92FF0E0E654F04E208130E0D6
:101E10009F5F90932620C90108958091252090917D
:101E20002620891B990B0895CF92DF92EF92FF92A3
:101E30000F931F93CF93DF937C01CB018A012091F5
:101E40004B20222389F0EB016B01C40ED51ECC156B
:101E5000DD0569F06991D701ED91FC910190F08168
:101E6000E02DC7010995F3CF642F0E94C30EC8016E
:101E7000DF91CF911F910F91FF90EF90DF90CF9066
:101E80000895CF93DF931F92CDB7DEB7698320917A
:101E90004B202223F9F020916E20203258F021E0CF
:101EA00030E0FC013383228390E080E00F90DF91EB
:101EB000CF91089580914C20E82FF0E0E35BFF4D37
:101EC000998190838F5F80934C2080936E2081E076
:101ED00090E0ECCF61E0CE0101960E94C30EF7CFF7
:101EE000682F86E293E20C94410F90E080E0089521
:101EF0008FB7F8948091B41F8FBF089561E0FC0103
:101F000084810E94BA088091B31F81111092B31F7F
:101F100008958EBD00000DB407FEFDCF8EB5089567
:101F20008FEF0C94890F0F931F93CF93DF93EC01E6
:101F30000E9471098B010E94900F8F3F69F00E94EF
:101F40007109601B710B6C177D07A8F380E0DF91AE
:101F5000CF911F910F91089581E0F9CF8CBD9DBD68
:101F60000895CF93DF93EC018091B31F811109C0D5
:101F700081E08093B31F80913223909133230E949C
:101F8000AE0F60E08C81DF91CF910C94BA088F92F4
:101F90009F92AF92BF92FF920F931F93CF93DF93C5
:101FA000EC01F62E49015A018E81882389F08F8138
:101FB00098859C012F5F3F4F38872F838230924056
:101FC00018F40E94900FF3CFCE010E947E0F1E8264
:101FD000CE010E94B10F8CE291E00E94930F8F2DF1
:101FE00080640E94890F08E110E0D501C401002E31
:101FF00004C0B695A795979587950A94D2F70E9445
:10200000890F08501109083F8FEF180771F785E90C
:10201000FF2021F028E087E8F2128FEF0E94890F5D
:1020200010E00E94900F8A8787FF04C01F3F11F0C5
:102030001F5FF7CFDF91CF911F910F91FF90BF905E
:10204000AF909F908F900895AF92BF92CF92DF9202
:10205000EF92FF920F931F93CF93DF93EC016901EF
:10206000C801820F931F8130924050F58E818823E2
:1020700079F088819981AA81BB8184179507A60789
:10208000B70731F48F819885C816D90608F042C089
:10209000488359836A837B838B85833039F089E059
:1020A000440F551F661F771F8A95D1F79A01AB0120
:1020B00061E1CE010E94C70F882389F083E08D8300
:1020C000CE010E947E0F80E0DF91CF911F910F9192
:1020D000FF90EF90DF90CF90BF90AF9008950E9457
:1020E00071095B010E94900F8A878F3F69F40E94FB
:1020F00071096A197B096D327140A0F38FE08D83FD
:10210000CE010E947E0FDCCF8E3F89F418861F829D
:1021100081E08E838F8198858C159D0550F40E94F7
:10212000900F8F819885019698878F83F3CF8DE0EC
:10213000E6CF6701E00EF11E0E94900FF601819339
:102140006F01EE15FF05C1F78F819885080F191FE4
:1021500018870F838985882319F001151240A0F094
:102160008E81882389F08F8198859C012F5F3F4F56
:1021700038872F838230924018F40E94900FF3CF5B
:10218000CE010E947E0F1E8281E09ECFCF92DF9211
:10219000EF92FF920F93CF93DF93EC01690182E1FD
:1021A000411551056105710599F08B85833039F032
:1021B00089E0440F551F661F771F8A95D1F79A0152
:1021C000AB0168E1CE010E94C70F882319F084E0BB
:1021D0008D832DC08EEF0E94890F76018EEFD81A65
:1021E000F70181917F010E94890FEC14FD04C1F772
:1021F0008FEF0E94890F8FEF0E94890F0E94900F2E
:102200008A878F71853071F4011116C0CE010E944A
:102210007E0F81E0DF91CF910F91FF90EF90DF90E3
:10222000CF90089581E18D83CE010E947E0FCE0173
:102230000E947E0F80E0EECF88E592E00E94930F2F
:10224000811102C085E1C4CF20E030E0A9016DE03A
:10225000CE010E94C70F882311F084E1B9CF0E94FC
:10226000900F8111FACFD2CF0F934091B61F5091AA
:10227000B71F6091B81F7091B91F411551056105D5
:10228000710599F0082F27E830E28091872290911C
:1022900088220E94C610882349F01092B61F10921F
:1022A000B71F1092B81F1092B91F81E00F910895C7
:1022B0000F93CF93C82F8091B51F811105C0C1E046
:1022C0008C2FCF910F9108954091240150912501B9
:1022D00060912601709127010C2F27E830E2809150
:1022E0008722909188220E94C610811102C0C0E00E
:1022F000E7CFCC2321F381E00E9434118823B9F386
:102300001092B51FDDCF8F929F92AF92BF92EF9246
:10231000FF920F931F93CF934B015C01C42F8091C9
:10232000240190912501A0912601B09127018815E3
:102330009905AA05BB0551F181E00E945811811150
:102340000BC080E0CF911F910F91FF90EF90BF9055
:10235000AF909F908F90089587E8E82E80E2F82E46
:1023600000E012E030E020E0B501A4018091872276
:10237000909188220E942410882319F380922401CE
:1023800090922501A0922601B09227014091B51F9D
:102390004C2B4093B51F81E0D5CF8F929F92AF9287
:1023A000BF92CF92DF92EF92FF92CF9324E333E27A
:1023B0003093882220938722882309F46DC040E05F
:1023C00060E070E0CB010E94831181110BC080E0BE
:1023D000CF91FF90EF90DF90CF90BF90AF909F9004
:1023E0008F900895809145228F7789F780915122AF
:1023F00090915222A0915322B0915422843691059B
:10240000A105B10520F3C0904D22D0904E22E0905E
:102410004F22F0905022C114D104E104F104B9F22A
:1024200040E0C701B6010E948311882381F28091A8
:102430009220909193208115924049F6A091972087
:10244000AA2329F26091952070919620611571055B
:1024500009F4BDCF20919420222309F4B8CFA09392
:1024600052232093442390E080E030E0E1E0F0E06C
:10247000C82FAF01082E02C0440F551F0A94E2F77F
:102480002417350769F041E0480F0196893091051E
:1024900079F740934D239BCFC12CD12C7601C0CF2F
:1024A00080934D2320919D2030919E2050E040E06C
:1024B0002115310541F42091AB203091AC204091A1
:1024C000AD205091AE202093452330934623409376
:1024D00047235093482346015701860E971EA11C9F
:1024E000B11C8092532390925423A0925523B09212
:1024F0005623E0919820F0919920F0935923E0938E
:102500005823B0E00E94374EDC01CB01880D991DA5
:10251000AA1DBB1D80935A2390935B23A0935C2339
:10252000B0935D2325E0EE0FFF1F2A95E1F7E15000
:10253000FE4FEF2FFF27E6958E0F9F1FA11DB11DA8
:1025400080934E2390934F23A0935023B093512315
:1025500080909A2090909B20B12CA12C8114910402
:1025600041F48090A7209090A820A090A920B0903E
:10257000AA20C81AD90AEA0AFB0AC80CD91CEA1C04
:10258000FB1C04C0F694E794D794C794CA95D2F77D
:10259000C0924923D0924A23E0924B23F0924C23DD
:1025A00085EFC8168FE0D806E104F10428F48CE02A
:1025B0008093572381E00CCF80E125EFC2162FEFE7
:1025C000D206E104F104A0F38091B3209091B420ED
:1025D000A091B520B091B62080935A2390935B23AD
:1025E000A0935C23B0935D2380E2E2CFCF93DF938F
:1025F000EC016E857F858889998941E00E9483116D
:10260000882351F08A8920E2829FC00111248957D2
:102610009F4DDF91CF91089590E080E0FACF4F92E7
:102620005F926F927F928F929F92AF92BF92CF9262
:10263000DF92EF92FF920F931F93CF93DF93EC0102
:10264000423051056105710590F480E0DF91CF9132
:102650001F910F91FF90EF90DF90CF90BF90AF90C0
:102660009F908F907F906F905F904F900895898595
:102670009A85AB85BC850196A11DB11D8417950770
:10268000A607B70710F3CB88DC88ED88FE888F8912
:10269000803109F042C0BB27A72F962F852F480114
:1026A00059012A013B01C80ED91EEA1EFB1E80916A
:1026B000240190912501A0912601B0912701C8160F
:1026C000D906EA06FB0699F58F898031C1F5B30179
:1026D000A201552766277727440F551F49575F4D9D
:1026E000FA01918280828091B51F81608093B51F2D
:1026F0008A89823080F08D819E81AF81B8858C0D72
:102700009D1DAE1DBF1D8093B61F9093B71FA09354
:10271000B81FB093B91F81E099CFDB01CA01E7E090
:10272000B695A79597958795EA95D1F7B8CF40E0EC
:10273000C701B6010E9483118111C6CF86CFB301B4
:10274000A2014F77552766277727440F551F440F5F
:10275000551F49575F4DFA0180829182A282B38250
:10276000C2CF8F929F92AF92BF92CF92DF92EF92A1
:10277000FF920F931F93CF93DF93FC018185928586
:10278000A385B4850196A11DB11D84179507A607E1
:10279000B70770F480E0DF91CF911F910F91FF9008
:1027A000EF90DF90CF90BF90AF909F908F90089563
:1027B00083889488A588B6888789803189F5BB2766
:1027C000A72F962F852FE9016A017B018F01BC019C
:1027D000CD01680D791D8A1D9B1D8090240190906C
:1027E0002501A0902601B090270186169706A8061D
:1027F000B90601F5F8018789803111F5DD24EE2451
:10280000FF24F601EE0FFF1FE957FF4D80819181F4
:10281000B0E0A0E088839983AA83BB8381E0BBCF2B
:10282000DB01CA01C7E0B695A79597958795CA952C
:10283000D1F7C9CF40E00E9483118111DBCFAACF2D
:10284000E894C7F8DD24EE24FF24F601EE0FFF1F05
:10285000EE0FFF1FE957FF4D80819181A281B38167
:10286000BF70D8CF4F925F926F927F92AF92BF921C
:10287000CF92DF92EF92FF920F931F93CF93DF934C
:1028800000D000D0CDB7DEB78C0149835A836B836B
:102890007C835901C12CD12C7601412C82E0582E29
:1028A000612C712C49815A816B817C819E012F5F43
:1028B0003F4FC8010E94B113882339F1F801858583
:1028C000A301920104C0220F331F441F551F8A9594
:1028D000D2F7DA01C901C80ED91EEA1EFB1E4981D2
:1028E0005A816B817C818789803111F188EF9FEF5C
:1028F000AFEFBFE0481759076A077B0798F2F50169
:10290000C082D182E282F38281E00F900F900F901B
:102910000F90DF91CF911F910F91FF90EF90DF907B
:10292000CF90BF90AF907F906F905F904F90089541
:1029300088EF9FEFA0E0B0E0DDCFCF93DF93FC0105
:102940002581222321F080E0DF91CF910895EC01D1
:1029500080915723803159F582E08583178A108E44
:10296000118E128E8091582390915923B0E0A0E0EF
:1029700025E0880F991FAA1FBB1F2A95D1F7838BCB
:10298000948BA58BB68B80E493E29C8F8B8F81E038
:102990008C831E821F82188619861A861B861C86C7
:1029A0001D861E861F86188A198A1A8ACDCF803204
:1029B00051F683E0858340915A2350915B236091C7
:1029C0005C2370915D23478B508F618F728F9F01C5
:1029D0002D5E3F4F80E493E20E9432148111D3CFE9
:1029E000B2CF8F929F92AF92BF92CF92DF92EF922F
:1029F000FF920F931F93CF93DF93EC018D81811191
:102A00000EC080E0DF91CF911F910F91FF90EF906A
:102A1000DF90CF90BF90AF909F908F9008950B89DB
:102A20001C892D893E89041715072607370748F3A7
:102A30004A015B01823031F48A869B86AC86BD8672
:102A400081E0E0CF81149104A104B10449F41E8215
:102A50001F82188619861A861B861C861D86F0CF53
:102A60000A851B852C853D85EB8DFC8D858590E049
:102A70000996B901A8014150510961097109082E4F
:102A800004C076956795579547950A94D2F77501D6
:102A90006401E1E0CE1AD108E108F10804C0F6941F
:102AA000E794D794C7948A95D2F7C416D506E6065C
:102AB000F70620F0012B022B032B11F58F89988D3F
:102AC000A98DBA8D8E839F83A887B9878E010A5FEF
:102AD0001F4FC114D104E104F10409F4ADCF4E81BC
:102AE0005F816885798598018B8D9C8D0E94B113DB
:102AF00091E0C91AD108E108F1088111EACF81CF2C
:102B0000C41AD50AE60AF70AE1CF3F924F925F92C4
:102B10006F927F928F929F92AF92BF92CF92DF92ED
:102B2000EF92FF920F931F93CF93DF93CDB7DEB752
:102B30002C970FB6F894DEBF0FBECDBF5C01DC0151
:102B40005B968D909C905C9716964D905D906D90E5
:102B50007C901997411451046104710409F468C010
:102B6000BFEF4B1A5B0A6B0A7B0A312CF40181859B
:102B70009285A385B4859C01AD012F5F3F4F4F4FD8
:102B80005F4F29873A874B875C87730162011D82FB
:102B90001E821F821886F40181859285A385B485E3
:102BA0002D813E814F815885281739074A075B07D9
:102BB00008F056C089859A85AB85BC858C159D0526
:102BC000AE05BF0550F482E0C82ED12CE12CF12CCB
:102BD00092E0492E512C612C712C9E012F5F3F4FAA
:102BE000B701A601C4010E94B1138823C9F18981EC
:102BF0009A81AB81BC81892B8A2B8B2B09F1260111
:102C000037019FEF491A590A690A790A2D813E81D5
:102C10004F8158852F5F3F4F4F4F5F4F2D833E832E
:102C20004F8358873FEFC31AD30AE30AF30AB3CF9F
:102C3000F40140805180628073803324339496CFB6
:102C4000C414D504E604F70409F70FEF1FEF2FEFC4
:102C50003FE0B701A601C4010E940F13811119C002
:102C600080E02C960FB6F894DEBF0FBECDBFDF918B
:102C7000CF911F910F91FF90EF90DF90CF90BF9079
:102C8000AF909F908F907F906F905F904F903F900C
:102C90000895D50116964D915D916D917C9119978E
:102CA000411551056105710539F097018601C4018F
:102CB0000E940F138823A1F2D5011696CD92DD92C2
:102CC000ED92FC921997332051F0D701C60101967D
:102CD000A11DB11DF40180839183A283B383F5010B
:102CE0008789908DA18DB28D892B8A2B8B2B39F4FE
:102CF0008481C78AD08EE18EF28E80688483F5014C
:102D000084818062848381E0ACCF2F923F924F9286
:102D10005F926F927F928F929F92AF92BF92CF926B
:102D2000DF92EF92FF920F931F93CF93DF93EC010B
:102D30005B012A018D81811115C08FEF9FEFDF911B
:102D4000CF911F910F91FF90EF90DF90CF90BF90A8
:102D5000AF909F908F907F906F905F904F903F903B
:102D60002F9008958C8180FFE8CF0B891C892D89D5
:102D70003E894A855B856C857D85C201B0E0A0E017
:102D800068017901C41AD50AE60AF70AC816D906F5
:102D9000EA06FB0618F42801441A550A42011E01EE
:102DA00026E0220E311C8114910409F4B3C04A8537
:102DB0005B856C857D856A0181E0D8228B8D9C8D39
:102DC0008A019B01E9E03695279517950795EA95C5
:102DD000D1F7ED81E230E1F5FC01628D738D848DD8
:102DE000958D600F711F821F931F612C22E0722E40
:102DF0006C187D088614970408F434012C8126FD94
:102E000004C06114F2E07F0671F400912401109176
:102E10002501209126013091270106171707280761
:102E2000390709F053C040E00E948311882309F458
:102E300084CFC60189579F4DD5019C01260D371DB2
:102E4000FC012E173F0709F460C041914D93F9CF63
:102E5000FC0174807A947022C114D10471F4711051
:102E60000CC0452B462B472B39F58F89988DA98DA2
:102E7000BA8D8E839F83A887B987EB8DFC8D6E8179
:102E80007F8188859985625071098109910925851D
:102E900004C0660F771F881F991F2A95D2F70685F1
:102EA000178520893189600F711F821F931F670D5D
:102EB000711D811D911D99CF4E815F816885798536
:102EC00091010E94B1138111D8CF37CF75018301D1
:102ED0009601AB01BC0180918722909188220E94CB
:102EE0002410882309F429CFA60CB71C8A859B855A
:102EF000AC85BD85860D971DA11DB11D8A879B8759
:102F0000AC87BD87861897084ECF281B390BA20EB9
:102F1000B31EECCFC20113CF1F93CF93DF93FC01FD
:102F20002581222371F1162FEC01848187FF1EC0B9
:102F3000CF010E94F612FC01892B19F18D8182309C
:102F400040F48B899C89AD89BE89848F958FA68F2B
:102F5000B78F8F89988D938F828F8F89988DA98D48
:102F6000BA8DB58BA48B8C818F778C83111103C0A4
:102F70008C818F7E8C83812FDF91CF911F910C9458
:102F8000581180E0DF91CF911F910895FF920F9328
:102F90001F93CF93DF93EC018D81813041F090E05E
:102FA00080E0DF91CF911F910F91FF9008958C8168
:102FB00081FFF5CF82FD1BC00091872210918822EE
:102FC000C8010E94B10F0E94900FF82EC8010E9404
:102FD0007E0F8FEFF812E3CF8C8185FF1BC060E07E
:102FE000CE010E948C178C818F7D8C83D8CF4B892A
:102FF0005C896D897E898A859B85AC85BD858417B2
:103000009507A607B707C1F2CE010E94F1148111FE
:10301000D3CFC5CF4091B61F5091B71F6091B81F55
:103020007091B91F452B462B472B21F080E00E9461
:103030003411B5CF80618C832A853B85317080E067
:1030400092E0821B930BADCFCF93DF93EC0161E055
:103050000E948C17882311F01D8281E0DF91CF91AF
:1030600008958F929F92AF92BF92CF92DF92EF928C
:10307000FF92CF93DF93EC010E94851581110CC064
:1030800080E0DF91CF91FF90EF90DF90CF90BF90E5
:10309000AF909F908F900895EB8DFC8DCE80DF8058
:1030A000E884F98482E0C81AD108E108F10885852E
:1030B00004C0CC0CDD1CEE1CFF1C8A95D2F7868563
:1030C0009785A089B189C80ED91EEA1EFB1E84818E
:1030D00046015701880E911CA11CB11CC814D904CB
:1030E000EA04FB04F9F081E0881A9108A108B1080C
:1030F00081E00E945811882319F2E7E8F0E211926A
:1031000082E2E738F807D9F78092240190922501EE
:10311000A0922601B09227018091B51F8160809313
:10312000B51FDCCFEB8DFC8D258580E092E0A0E023
:10313000B0E004C0880F991FAA1FBB1F2A95D2F7C1
:103140004B895C896D897E89840F951FA61FB71FE7
:103150008B8B9C8BAD8BBE8B81E093CF2F923F925C
:103160004F925F926F927F928F929F92AF92BF9297
:10317000CF92DF92EF92FF920F931F93CF93DF9343
:1031800000D000D01F92CDB7DEB77C015B01342E9A
:103190005D83DC0115968C911597813009F0CEC0C6
:1031A00014962C9021FECAC022FCB4C0C32CDD8032
:1031B00022947FE027222094B22DB1702B2ED701CC
:1031C0001A964D915D916D917C911D97C114D1041A
:1031D00009F428C15B968D919C915C97FC017480E9
:1031E0007A948A019B0169E0369527951795079592
:1031F0006A95D1F770228A011170711020C00115F3
:103200001105E9F416964D915D916D917C91199798
:10321000411551056105710509F099C057968D91C9
:103220009D910D90BC91A02D0097A105B10509F0CD
:10323000B0C0C7010E948515882309F47FC080E0D3
:1032400092E0801B910B46018C159D0508F44C0102
:10325000D7015B964D915C915C9716968D919D91EF
:103260000D90BC91A02D0297A109B109FA01258505
:1032700004C0880F991FAA1FBB1F2A95D2F7468545
:10328000578560897189840F951FA61FB71F9C0100
:10329000AD01270D311D411D511D29013A01811438
:1032A00032E0930609F07BC08091240190912501C2
:1032B000A0912601B091270184159505A605B705B3
:1032C00059F48FEF9FEFDC01809324019093250147
:1032D000A0932601B0932701022D9501B301A2010D
:1032E00080918722909188220E94C610882331F114
:1032F0009EEFB91AC818D908F70182859385A4856D
:10330000B585880D991DA11DB11D82879387A4875E
:10331000B58755CFF70143895489658976898285B8
:103320009385A485B585481759076A077B0709F473
:103330003DCFC7010E94F114811138CF81E090E0A8
:10334000D70113969C938E93129780E007C09E013D
:103350002F5F3F4F0E94B113811102C090E079C0EE
:1033600089819A81AB81BC81F701238D348DF9016C
:10337000278948EF5FEF60E070E0203121F048EFEF
:103380005FEF6FEF7FE084179507A607B70708F098
:1033900050CFF70186839783A087B18750CF01155F
:1033A000110599F5D7011A964D915D916D917C911A
:1033B0001D9753968D919D910D90BC91A02D48170E
:1033C00059076A077B0708F181E00E94581188239A
:1033D00009F4B4CF40922401509225016092260155
:1033E000709227018091B51F81608093B51FC8013D
:1033F00089579F4DD5019C01280D391DFC012E17C1
:103400003F0759F04D914193FACF41E0C301B2011A
:103410000E9483118111EBCF91CF281B390BA20E93
:10342000B31E68CFF70183899489A589B68984176B
:103430009507A607B70738F48481438B548B658BB7
:10344000768B80688483F701848183FD1AC0832D85
:103450009D810F900F900F900F900F90DF91CF9163
:103460001F910F91FF90EF90DF90CF90BF90AF90A2
:103470009F908F907F906F905F904F903F902F9094
:10348000089561E0C7010E948C17882309F456CF84
:10349000DECFCF93DF931F92CDB7DEB7698341E0D4
:1034A00050E0BE016F5F7F4F0E94AE180F90DF911A
:1034B000CF910895FC01DB0112968D919C91139799
:1034C0009383828380E991E09183808314968C9129
:1034D0001497848315968C911597858316964D9134
:1034E0005D916D917C9119974683578360877187B1
:1034F0001A964D915D916D917C911D9742875387EE
:10350000648775871E964D915D916D917C91519761
:1035100046875787608B718B52968C915297828B1E
:1035200053964D915D916D917C915697438B548B41
:10353000658B768B57964D915D916D917C915A97E5
:10354000478B508F618F728F5B968D919C91948F7A
:10355000838F08950895FC01818D928D009719F055
:1035600061E00C948C170895DC015996ED91FC9163
:103570003097B9F083899489A589B68942855385A6
:1035800064857585841B950BA60BB70B811520E808
:103590009207A105B10538F08FEF9FE7A0E0B0E0FA
:1035A000089590E080E00895DC0159968D919C91FA
:1035B000009739F0DC01ED91FC910480F581E02D5C
:1035C000099490E080E00895CF93DF93EC01E98DBA
:1035D000FA8D309749F481E090E09B838A8390E0F4
:1035E00080E0DF91CF91089513821282898D9A8DA8
:1035F0000E94AE18E98DFA8D22813381232B59F771
:10360000F0CFCF93DF931F92CDB7DEB76983DC0194
:10361000ED91FC910280F381E02D41E050E0BE018C
:103620006F5F7F4F09950F90DF91CF910895CF93F2
:10363000DF931F92CDB7DEB741E050E0BE016F5F70
:103640007F4F0E948516019731F4898190E00F9099
:10365000DF91CF9108958FEF9FEFF9CF1F93CF9315
:10366000DF93FC012581223030F490E080E0DF918F
:10367000CF911F910895EC0142855385648575852E
:1036800085E076956795579547958A95D1F7142FDC
:103690001F70CF010E94171B97FDE7CF8A859B857E
:1036A000AC85BD854F96A11DB11D8A879B87AC87D0
:1036B000BD87F0E21F9FC001112489579F4DD7CFCE
:1036C000FC01818D928D009711F00C94171B8FEFE8
:1036D0009FEF08950F931F93CF93DF93EC01898D94
:1036E0009A8D10E000E0009799F00E94171B8C0162
:1036F0000F3F100769F0898D9A8DFC014285538533
:103700006485758541505109610971090E94F11460
:10371000C801DF91CF911F910F910895809175207D
:103720009091762020917B2028171906C1F41092E1
:10373000B21F1092B11F80918120809382208DEB67
:103740009BE190931E2080931D2080917520909185
:10375000762001969093762080937520089520918D
:1037600075203091762080917C2090917D202817C3
:10377000390759F783E29DE0E4CF3091840020912E
:1037800080202A50231B2350F0F72D5F19F02A9533
:1037900011F001C00000E0911F20F0912020099558
:1037A0009091822080918120911138C08093822055
:1037B00020917F204091B11F5091B21F240F352FCF
:1037C000311D3093B21F2093B11F2091752030918D
:1037D00076202F5F3F4F082E000C990B01966091C9
:1037E0007E20689FA001699F500D112480917B204D
:1037F000840F952F911D2817390731F48EE89BE12E
:1038000090931E2080931D208091752090917620AA
:10381000019690937620809375200895915090930F
:103820008220D3CF089590917F20E82FE695E695EA
:10383000E695F0E0699FE00DF11D112420918420B0
:1038400030918520E20FF31F90818770413051F451
:1038500020E830E002C0359527958A95E2F7922B53
:1038600090830895411109C02FE73FEF02C03595BD
:1038700027958A95E2F79223F3CF20E830E002C043
:10388000359527958A95E2F79227EACF20917F20F8
:1038900098E0299F900111248217130634F4909127
:1038A0007E20691710F40C94131C0895CF93DF93B6
:1038B000FB01DA016417750739F4422F682F8E2F48
:1038C000DF91CF910C94461C4617570720F4AB01AB
:1038D0005527FD01DA01AF0147705527CFEFD0E042
:1038E000BE0102C0759567954A95E2F7AB01362F88
:1038F00093E0F695E7959A95E1F760917F20869F92
:10390000B0011124E60FF71FCD018770992702C07F
:10391000D595C7958A95E2F79C2F909553E0B6957B
:10392000A7955A95E1F7A60FB71FEA17FB0719F4F9
:10393000392F342390E0213001F5AF014F5F5F4F05
:1039400060916F2070917020E60FF71F8081382BF7
:1039500030838FEFE0916F20F0917020E40FF51F1E
:103960004A175B0720F44F5F5F4F8083F3CF80815E
:10397000982B9083DF91CF91089521111EC0AF0144
:103980004F5F5F4F60916F2070917020E60FF71FBF
:103990003095808138233083E0916F20F091702042
:1039A000E40FF51F4A175B0720F44F5F5F4F10824B
:1039B000F3CF909580819823DCCF2230D9F6AF01E8
:1039C0004F5F5F4F60916F2070917020E60FF71F7F
:1039D000808138273083E0916F20F0917020E40FD0
:1039E000F51F80814A175B0728F44F5F5F4F809572
:1039F0008083F1CF9827BDCFCF92DF92EF92FF92D5
:103A00000F931F93CF93DF93D42FC62FE62EF12C65
:103A100097E0E90EF11C082F10E0680185E0C80E60
:103A2000D11CCE151F0444F42D2FA601B8018C2FF4
:103A30000E94561CCF5FF5CFDF91CF911F910F9160
:103A4000FF90EF90DF90CF9008952F923F924F928A
:103A50005F926F927F928F929F92AF92BF92CF921E
:103A6000DF92EF92FF920F931F93CF93DF9300D0DB
:103A700000D0CDB7DEB7962F622F202FE82EF12C85
:103A800000917F20C02ED12CF60153E0EE0FFF1FD6
:103A90005A95E1F7EE15FF050CF416C130917E2022
:103AA000391708F411C1442E512CE415F5050CF416
:103AB0000BC1361708F408C184137FC070E0A92F2A
:103AC000B0E06A177B07D1F4422F692F0F900F9057
:103AD0000F900F90DF91CF911F910F91FF90EF907A
:103AE000DF90CF90BF90AF909F908F907F906F901E
:103AF0005F904F903F902F900C94461C6A177B0765
:103B000028F0362F972FBD01A32FB92F982F97702C
:103B1000E0E8F0E002C0F595E7959A95E2F73E2FD0
:103B2000869586958695C69EA001C79E500DD69E09
:103B3000500D1124840F952F911D213091F4A6175B
:103B4000B70708F4C1C0E0916F20F0917020E80F32
:103B5000F91F2081232B20838C0D9D1D6F5F7F4FCC
:103B6000EECF211115C05E2F5095A617B70708F4A8
:103B7000ABC020916F2030917020280F391FF901C0
:103B80004081452340838C0D9D1D6F5F7F4FEDCF9E
:103B9000223009F099C0A617B70708F495C0E09144
:103BA0006F20F0917020E80FF91F208123272083D8
:103BB0008C0D9D1D6F5F7F4FEECF96131BC0A20132
:103BC000B701892F0F900F900F900F90DF91CF9139
:103BD0001F910F91FF90EF90DF90CF90BF90AF902B
:103BE0009F908F907F906F905F904F903F902F901D
:103BF0000C94561CC92ED12C481708F050C08701D0
:103C00000419150928018FEF462F50E05C834B8380
:103C1000691708F048C08601041B150B1C830B8331
:103C20009FEF0B811C81401651060CF444C04B8160
:103C30003C815C824B82442E532E19822A83440C91
:103C4000551C82012B813C81021B130B1901220C94
:103C5000331C912C812C692E990F7708A82E880F80
:103C6000BB084B815C814815590574F14A816C2D64
:103C70008E2D0E94131C17FD07C059815130F1F49D
:103C8000EA0CFB1C0219130969816130D1F4C60CDE
:103C9000D71C040D151D7FEF871A970AE2CF4E1827
:103CA0005F0881E0B1CF0B811C810C191D091C83B9
:103CB0000B8391E0B6CF11E01983C0CFC60CD71C9F
:103CC000E1CFEA0CFB1CE5CF0F900F900F900F9007
:103CD000DF91CF911F910F91FF90EF90DF90CF90E8
:103CE000BF90AF909F908F907F906F905F904F901C
:103CF0003F902F90089540912E2020912D2090915B
:103D0000B01F241306C020932D209093B01F80E095
:103D100008952F5F2D3208F020E0E22FF0E0ED57FC
:103D2000F04EE081EE2379F3E03F11F49160E9CFAA
:103D3000E03E11F49260E5CF90FF09C0E23119F442
:103D40009B7F9C7FDECFE935E1F7977FFACFE231A9
:103D500011F49460D6CFE93511F49860D2CF392FA1
:103D60003C7F91FF11C0EA54E43310F0932FC9CF88
:103D7000F0E0EC5CFE4F8081932F882311F22093BA
:103D80002D203093B01F08959C7039F0E43870F7FF
:103D9000F0E0EF5BFB4F8491EFCFE43838F7F0E0D1
:103DA000E354FC4FF8CF80918620882331F01092A5
:103DB0008620082E000C990B08950E947B1E81110D
:103DC000F8CF8FEF9FEF08958091C00087FF13C059
:103DD00080912E208F5F8D3208F080E090912D2011
:103DE000981749F09091C600E82FF0E0ED57F04E9B
:103DF000908380932E2008951F93CF93DF93EC013F
:103E0000162F81E080934B2080E580936D201092E7
:103E10004C2010926E208D2F90E00E94700FCE01EA
:103E200099270E94700F612F86E293E20E94410F52
:103E300081E00E947F0665E070E080E090E0DF9125
:103E4000CF911F910C943E0982EA94E09093821FD7
:103E50008093811F909331208093302080912201A4
:103E6000909123018E559B4F9093A1048093A004C1
:103E70009C012253310930939F0420939E0488565D
:103E800091099093332080933220089590ED980FFC
:103E90009A3090F0982F9F7D91549A3168F08F3529
:103EA00059F08B3249F08E3239F021E090E08E37B4
:103EB00009F020E0822F089581E090E00895EF92CC
:103EC000FF920F931F93CF93DF9310928704C091BB
:103ED0009204D09193048E01F88021968F2D0E9438
:103EE000461F892BC1F3F1100FC010939304009368
:103EF000920481E080938704C801DF91CF911F91E4
:103F00000F91FF90EF9008957E012196F701808137
:103F10000E94461F892BC1F7F0929304E09292040D
:103F20000E151F0511F0F7011082F801808188231A
:103F300001F3E2CFCF93DF9300D000D01F92CDB733
:103F4000DEB7FE013196BE01635071094E2F3F2F3F
:103F5000282F2F702A30C0F4205D238324E096950B
:103F600087952A95E1F731976E177F0789F71D82AC
:103F7000842F932F0E943C060F900F900F900F906C
:103F80000F90DF91CF910895295CE7CFE091302029
:103F9000F0913120329690E081918A30A9F0891712
:103FA000D1F3823269F0873269F09111F5CF2FE9B0
:103FB000280F2A3188F7DF01119780528C93ECCFBC
:103FC00092E2EACF97E2E8CF08958091811F909125
:103FD000821F409130205091312060918D0470916A
:103FE0008E044817590751F0FC01208131812617B2
:103FF000370720F42281820F911DF3CF0895E091BD
:104000009204F09193042E2F9F2F81918032D9F347
:104010008930C9F3209392049093930408950E94E9
:10402000FF1FE0919204F091930490E080E05AE049
:104030003E2F2F2F419160ED640F6A30A8F489392B
:1040400069E1960738F030939204209393048FEF40
:104050009FEF0895589F9001599F300D1124C90179
:10406000C097840F911DE4CF309392042093930462
:104070000895CF93DF93EC011092880490E080E0E4
:10408000FE012491222371F14091920450919304F6
:10409000FA01E80FF91F2081FE013491231303C0B8
:1040A00001962196EDCF649130E020583F4F621782
:1040B000130659F40196840F951F909393048093EF
:1040C0009204DF91CF910C94FF1FFE018491219601
:1040D00087FFFBCF809188048F5F809388040E94C4
:1040E000FF1FCCCFDF91CF9108952F923F924F9237
:1040F0005F926F927F928F929F92AF92BF92CF9278
:10410000DF92EF92FF920F931F93CF93DF93CDB780
:10411000DEB7A0970FB6F894DEBF0FBECDBF6B0120
:104120007C01F7FE5BC08DE20E94EA05F094E0940A
:10413000D094C094C11CD11CE11CF11CC701B60174
:104140008E010F5F1F4F412C512C320118012AE0C4
:10415000822E912CA12CB12C730162012FEFC21A77
:10416000D20AE20AF20AA50194010E944A4EF8011D
:1041700061938F01B901CA0161157105810591052E
:1041800009F04DC010E000E0F201E01BF10BE20D80
:10419000F31D80818A3008F045C0805D0E94EA05E9
:1041A0000F5F1F4F0C151D0579F7A0960FB6F894F9
:1041B000DEBF0FBECDBFDF91CF911F910F91FF905A
:1041C000EF90DF90CF90BF90AF909F908F907F90B7
:1041D0006F905F904F903F902F900895C114D1043D
:1041E000E104F10409F0AACF80E3A0960FB6F89499
:1041F000DEBF0FBECDBFDF91CF911F910F91FF901A
:10420000EF90DF90CF90BF90AF909F908F907F9076
:104210006F905F904F903F902F900C94EA0526018D
:1042200037019ACF895CBACF8F929F92AF92BF929B
:10423000CF92DF92EF92FF920F931F93CF93DF9372
:1042400000D000D0CDB7DEB7FC018581813091F080
:1042500080E00F900F900F900F90DF91CF911F9102
:104260000F91FF90EF90DF90CF90BF90AF909F9015
:104270008F900895848181FFEBCF83899489A589EC
:10428000B689892B8A2B8B2B09F45FC07F0140E014
:1042900050E0BA01CF010E94F1148823C9F2F7015E
:1042A000C38CD48C8788908CA18CB28C82E090E0F7
:1042B000A0E0B0E0F60180839183A283B3839E01E6
:1042C0002F5F3F4FB501A401C6010E94B11388239F
:1042D00009F4BECF00E010E09801B501A401C601C9
:1042E0000E940F13882309F4B3CF89809A80AB8092
:1042F000BC80F6018789803119F188EF9FEFAFEF1D
:10430000BFE088169906AA06BB06C8F2F701178A0D
:10431000108E118E128E138A148A158A168A848141
:104320008068848361E0C7010E948C17882309F4A8
:104330008FCF40E050E0BA01C7010E94F11489CF4D
:1043400088EF9FEFA0E0B0E0DCCF81E082CFCF9399
:10435000DF93EC010E941421882371F0CE010E94AA
:10436000F612009749F025EEFC0120831D8281E0C2
:10437000DF91CF910C94581180E0DF91CF91089597
:10438000CF92DF92EF92FF921F93CF93DF93EC01D6
:1043900080E2689FF0011124E957FF4D93859171E8
:1043A00061F0842F827449F080E0DF91CF911F91FA
:1043B000FF90EF90DF90CF900895142F6A8B80913B
:1043C000240190912501A0912601B09127018E87AB
:1043D0009F87A88BB98BC488D588F12CE12C7601F6
:1043E000DD24CC24CF8AD88EE98EFA8E828D938DEF
:1043F000B0E0A0E0AC01BD014C295D296E297F2908
:104400004F8B588F698F7A8F83858871B1F4848D33
:10441000958DA68DB78D8B8B9C8BAD8BBE8B81E0E4
:104420008D831F701C831E821F82188619861A8630
:104430001B861C861D8681E0B8CF803109F0B4CF81
:104440009E012D5E3F4F8B8D9C8D0E9432148823E0
:1044500009F4AACF84E0E4CFCF93DF93EC0181E0AD
:1044600080934B2080E580936D2010924C20109219
:104470006E208D2F90E00E94700FCE0199270E9430
:10448000700F81E00E947F0680914A208111FCCF4D
:1044900081E080934A20809349209FEF90934820A9
:1044A0002AEB3FE13093472020934620109245208D
:1044B000109244208093432080914320806A80930F
:1044C000432080914220813021F51092422080913A
:1044D00043208093BB008091BC0083FDF8CF85EC26
:1044E0008093BC0080914A208130E1F38091452087
:1044F000811111C0809145201092262080932520A3
:10450000882359F086E293E20E94FA0EDF91CF9160
:10451000089585EEE5CF81E0EFCF8FEFF7CF9F9243
:10452000AF92BF92CF92DF92EF92FF920F931F93C1
:10453000CF93DF93CDB7DEB72B970FB6F894DEBFDE
:104540000FBECDBF8C01FC018581811115C0FE011C
:104550003196CE010C965F0130E23193E817F907EE
:10456000E1F7DA0130E087E09D91D92E992329F116
:104570009E3239F48A3011F480E0B9C038E08AE024
:10458000F3CFE5ECF4E04491442321F03196941309
:10459000FACFF2CF831780F34FED490F4E3560F716
:1045A0004FE9490F4A3118F440EED42ED90EF501E7
:1045B000E30FF11DD0823F5FD7CF89818032E1F2D6
:1045C000C22E7B01FB01838D948DF801948F838F24
:1045D000FB011682178210861186128613861486B6
:1045E0001586F70182859385A485B585438954890D
:1045F0006589768984179507A607B70790F525E0A2
:10460000B695A795979587952A95D1F7F82FFF70BE
:104610009F2EC7010E942E1B009709F4ADCFFC010D
:104620002081222341F0253E09F04EC0DD2029F0F3
:10463000DD24D394D6CFD1100EC0F801928A4091D8
:104640002401509125016091260170912701468730
:104650005787608B718BFC0180818111E9CFDD244C
:10466000D3948C2D8271823109F086CFDD2009F43C
:1046700050C0C8010E94F612009709F47DCF20E2D5
:10468000FC0111922A95E9F72BE0F501DC0101907C
:104690000D922A95E1F721E238E2FC01318B208B63
:1046A00040E058E057874687338B228B318F208F2D
:1046B000578B468B81E00E945811882309F45CCF08
:1046C0004C2DF801628910C04BE050E0BC01C501DF
:1046D0000E94AA50892B09F084CF8C2D80734C2D19
:1046E000692D803309F448CFC8010E94C0212B9660
:1046F0000FB6F894DEBF0FBECDBFDF91CF911F91F3
:104700000F91FF90EF90DF90CF90BF90AF909F9070
:104710000895F7018581823009F42ECFC7010E94E8
:104720003118882309F428CFF801128A87E890E22B
:10473000A6CF5F926F927F928F929F92AF92BF921D
:10474000CF92DF92EF92FF920F931F93CF93DF935D
:10475000CDB7DEB7C754D1090FB6F894DEBF0FBE90
:10476000CDBF5C013B0119A218A280E991E09F8FA7
:104770008E8F1BA21C821B829A8389831E8210E06B
:1047800000E06E018EE1C80ED11C8EE5E82E83E2BA
:10479000F82EF501E00FF11F80818F3211F40F5FC9
:1047A0001F4FD501A00FB11FFE01FB9690E080E0E6
:1047B0004F012D912F3249F0222339F00F5F1F4F07
:1047C000019621938C309105A1F7880D991DFC016C
:1047D0001082F501E00FF11F80818F3211F40F5F1D
:1047E0001F4FF501E00FF11F508041E0511040E0F4
:1047F00030E020E0B401C701F3010995811121C027
:10480000FEE5EF16F3E2FF06C1F480E0C95BDF4F7F
:104810000FB6F894DEBF0FBECDBFDF91CF911F91D1
:104820000F91FF90EF90DF90CF90BF90AF909F904F
:104830008F907F906F905F900895C7010E94241819
:10484000E4CF552091F021E0A401B701C6010E94F8
:104850008F22982E8EE5E81683E2F80681F0C701D4
:104860000E942418911010C0D0CF9EE5E91693E263
:10487000F90619F0C7010E94241881E0C7CF9920DA
:1048800021F2FE0131967F019E2D8F2D7601C92EDA
:10489000D82E7FCF6EE474E20C9499231F93CF93AC
:1048A000DF93CDB7DEB76D970FB6F894DEBF0FBEBE
:1048B000CDBFAB011C821B8220E931E03A83298302
:1048C0001E8221E0BC01CE0101960E948F2211E0E0
:1048D00081110CC010E0812F6D960FB6F894DEBFE9
:1048E0000FBECDBFDF91CF911F910895CE010196EC
:1048F0000E942418F0CFCF93DF93CDB7DEB76D972A
:104900000FB6F894DEBF0FBECDBF442309F453C0E9
:10491000AB01BC011C821B8280E991E09A838983F0
:104920001E8221E0CE0101960E948F22882339F059
:104930008E81843071F090E081E0911101C080E0BF
:104940006D960FB6F894DEBF0FBECDBFDF91CF914D
:1049500008951F82188619861A861B861C861D8656
:104960001E864B855C856D857E858C899D89AE898B
:10497000BF89481759076A077B0790F4CE01019653
:104980000E942E1B0097B9F2FC012081222341F0E6
:10499000253E39F32E3229F3838583FDE2CFCBCF39
:1049A00081E08E838D8182608D83CE0101960E948D
:1049B000A721982FC1CF81E0C3CFCF93DF93CDB78D
:1049C000DEB76D970FB6F894DEBF0FBECDBF4423A0
:1049D00011F1AB01BC011C821B8280E991E09A833A
:1049E00089831E8222E0CE0101960E948F228823B5
:1049F00021F0CE0101960E94A72191E0811101C012
:104A000090E0892F6D960FB6F894DEBF0FBECDBF34
:104A1000DF91CF91089591E0F4CF8F929F92AF9262
:104A2000BF92EF92FF920F931F93CF93DF93CDB777
:104A3000DEB7ED970FB6F894DEBF0FBECDBF8C0189
:104A40007B011CA21BA280E991E09AA389A31EA26C
:104A5000C8010E944E248111A0C023E3A701B80120
:104A6000CE0181960E948F22811116C090E081E0D4
:104A7000911101C080E0ED960FB6F894DEBF0FBE35
:104A8000CDBFDF91CF911F910F91FF90EF90BF901D
:104A9000AF909F908F90089581E08DA384E08EA3C6
:104AA000CE0181960E943118882301F361E0CE0186
:104AB00081960E948C178823C9F2CE0181960E94AC
:104AC000F612FC01892B91F280E1838780E2DE01FE
:104AD000119601900D928A95E1F7FE013296CE0172
:104AE0000C9620E22193E817F907E1F78EE2F82E01
:104AF000F982ECADFDAD68AD79AD8AAD9BAD62508C
:104B0000710981099109258504C0660F771F881FE7
:104B1000991F2A95D2F786849784A088B188680D5A
:104B2000791D8A1D9B1D41E00E948311882309F491
:104B30009DCF80E2FE013196A7E8B0E201900D9290
:104B40008A95E1F7FA82F80185818250823000F17E
:104B50004789508D618D728DCA019B013E8B2D8BD3
:104B60009C8F8B8F80E2FE013196A7EAB0E2019024
:104B70000D928A95E1F780E490E0A0E0B0E08BA789
:104B80009CA7ADA7BEA781E00E945811982F6FCFB8
:104B900090E080E030E020E0E1CF81E06CCFCF9387
:104BA000DF93EC01898D9A8D009741F00E942418C3
:104BB000898D9A8D0E942E4A1A8E198EDF91CF917F
:104BC0000895EF92FF920F931F93CF93DF93EC0121
:104BD0007B018A011B821A8288EE93E0A0E0B0E09C
:104BE0008C839D83AE83BF838CE991E09983888316
:104BF0008DE190E00E9492499A8F898F009779F019
:104C00002DE1F701DC0101900D922A95E1F74CE0CE
:104C100050E0B801CE010C960E94DD50188EDF9155
:104C2000CF911F910F91FF90EF9008952F923F9297
:104C30004F925F926F927F928F929F92AF92BF92AC
:104C4000CF92DF92EF92FF920F931F93CF93DF9358
:104C5000CDB7DEB7C756D1090FB6F894DEBF0FBE89
:104C6000CDBF5C013B01A6964FAFA69719A218A233
:104C700080E991E09F8F8E8F1BA21C821B829A83FA
:104C800089831E824E018EE1880E911CC4010E9410
:104C90009D1463018E010F5F1F4F240118016FE205
:104CA00070E0C6010E94C250009709F459C0F60195
:104CB00020812F3271F4FFEFCF1ADF0A902F812F5E
:104CC0008201492E582E942D852D2801092F182F49
:104CD000E6CF8C198D3008F08CE0E82EF12CA7017E
:104CE000B601CE01885A9F4F0E94DD50E8E5F0E002
:104CF000EC0FFD1FEE0DFF1D1082C8010E9424184D
:104D000021E0AE01485A5F4FB201C8010E948F22D4
:104D1000811120C01EAE1DAE80E991E09CAF8BAF2B
:104D200021961FAE2197A896EEADFFADA8976E0E07
:104D30007F1EF3018081811120C0BE01655C7F4F21
:104D4000C1010E945A1A4AEA51E0B101C5010E940C
:104D5000E12531C0CE0CDF1CC2010E942418B3CF64
:104D6000C60186199709A8969FAF8EAFA897B20182
:104D7000CE01CB960E945A1AD6CF19A218A280E96A
:104D800091E09F8F8E8F1BA221968FAD219781116D
:104D90002DC0F5011382128288EE93E0A0E0B0E00E
:104DA00084839583A683B7838CE991E09183808384
:104DB000128E118E1486C501C959DF4F0FB6F894B3
:104DC000DEBF0FBECDBFDF91CF911F910F91FF903E
:104DD000EF90DF90CF90BF90AF909F908F907F909B
:104DE0006F905F904F903F902F900895A6962FADB3
:104DF000A697A301BE01655C7F4FC4010E948F226C
:104E0000882339F2CE01CB960E942418A6968FAD46
:104E1000A6978670863039F449A95AA96BA97CA94E
:104E2000C4010E94F114B401C1010E945A1AA301E5
:104E30008CCF0C94024E682F80912820811129C0BC
:104E400080912A20813069F480919C0490919D0486
:104E50009C012F5F3F4F30939D0420939C040C9442
:104E60000A4E833069F480919C0490919D049C01CA
:104E70002F5F3F4F30939D0420939C040C94FC1EA5
:104E8000843021F48DE793E20C94011B862F0C945F
:104E9000EA0508958AE00E941B278DE00E941B27E7
:104EA00086E080932F208091722080932C2008959B
:104EB000CF93DF93EC01FE012491222329F0219668
:104EC00084910E941B27F7CFDF91CF9108950E9414
:104ED00058270C944A270F931F93CF93DF93809109
:104EE0002920833009F444C08430E1F0D1E0C1E0EE
:104EF000813009F050C080919C0490919D049C01E8
:104F00002F5F3F4F30939D0420939C040E941927EC
:104F1000C82FD0E02097C9F0CE01DF91CF911F912B
:104F20000F9108958DE793E20E94601BEC010A97B0
:104F300011F4CDE0D0E08DE793E20E94B41A892B02
:104F400059F78DE793E20E94CF2510922920109205
:104F5000282086EB93E00E946727809195048823A0
:104F600009F46EC01092950481E08093940468C0A7
:104F700080919C0490919D049C012F5F3F4F309342
:104F80009D0420939C040E942C22C82FD0E0CF3F88
:104F9000D10511F6DACF80918620811143C00E949D
:104FA0007B1E8093862081113DC00E947109009173
:104FB0009704109198042091990430919A04AB01C0
:104FC000BC01401B510B620B730B8091200190912F
:104FD0002101B0E0A0E0481759076A077B0778F085
:104FE000809196048D27809396040E9471096093A6
:104FF0009704709398048093990490939A048091F5
:1050000096048111C8CF80913420882341F080918B
:105010002F2042E060912C2086500E94FC1CC093FF
:105020009604B9CF0E94D31EEC0181E0C130D105B6
:1050300029F0C230D10509F06FCF82E080939B0444
:10504000CAE0D0E069CFCF93809130209091312099
:10505000029690939304809392040E946B278B3066
:10506000E1F39CF48830B4F08A30BCF380912F20B7
:1050700040E060912C2086500E94FC1C0E944A2730
:10508000E0919204F09193044AC0853131F39CF48D
:105090008D3061F3E0919204F091930420913220DD
:1050A0003091332022503109E217F307E1F588E00F
:1050B0000E941B27D2CFE0919204F09193048B3190
:1050C00059F18F3739F78091302090913120029635
:1050D000E817F90711F23197F0939304E0939204E3
:1050E00082EB93E00E945827109296040E94710967
:1050F00060939704709398048093990490939A0412
:10510000C0912F20C65040E060912C208C2F0E942F
:10511000FC1CC0932F20A1CF81E0809391048AE0F2
:105120008083CF9108958193F0939304E093920448
:1051300090912920911102C00E941B27809171201B
:105140008A5F80932F208091722080932C2085CFBE
:10515000CF93DF93E091A004F091A104D0E0C0E0F0
:105160002AE030E0B9010E947950805D8293CB0142
:1051700021960097B9F7F093A104E093A004E09181
:10518000A004F091A1048191F093A104E093A00404
:105190000E941B27219799F7DF91CF9108950F93D4
:1051A0001F93CF93DF93EC0197FF06C0D195C19574
:1051B000D1098DE20E941B27E091A004F091A10487
:1051C00010E000E02AE030E0CE01B9010E948D50ED
:1051D000805D8293EB010F5F1F4F1C161D06A4F329
:1051E000F093A104E093A004E091A004F091A10445
:1051F0008191F093A104E093A0040E941B27015029
:10520000110991F7DF91CF911F910F910895E091CE
:105210008B04F0918C04808191813396F0938C04FF
:10522000E0938B040E94CF2880E20E941B27E0912C
:105230008B04F0918C0480818A3061F00E941B27DE
:1052400080918B0490918C04019690938C048093B0
:105250008B04EDCF3196F0938C04E0938B040C9487
:105260004A271F93CF93DF93CDB7DEB761970FB671
:10527000F894DEBF0FBECDBF182F81E1ECEAF1E05C
:10528000DE01119601900D928A95E1F7E12FE295EA
:10529000EF7081E090E08C0F9D1F8E0F911DFC013F
:1052A00080810E941B27E12FEF7081E090E08C0F3E
:1052B0009D1F8E0F911DFC01808161960FB6F894A1
:1052C000DEBF0FBECDBFDF91CF911F910C941B2786
:1052D0000F931F93CF93DF93CDB7DEB761970FB6D0
:1052E000F894DEBF0FBECDBF8C0181E1ECEAF1E0A6
:1052F000DE01119601900D928A95E1F7F801EF2FEA
:10530000FF27E295EF7081E090E08C0F9D1FE80F82
:10531000F91F80810E941B27E12FFF27EF70FF27D5
:1053200081E090E08C0F9D1FE80FF91F80810E94A3
:105330001B27F80124E0F695E7952A95E1F7EF7031
:10534000FF2781E090E08C0F9D1FE80FF91F8081FF
:105350000E941B27F801EF70FF2781E090E08C0F7F
:105360009D1FE80FF91F808161960FB6F894DEBF8C
:105370000FBECDBFDF91CF911F910F910C941B27D2
:10538000CF92DF92EF92FF920F931F93CF93DF9311
:105390000091A0041091A104D0E0C0E02AE0C22E48
:1053A000D12CE12CF12CA70196010E944A4E605DA0
:1053B000F80162938F01B901CA0121966115710547
:1053C0008105910581F7F093A104E093A004E09199
:1053D000A004F091A1048191F093A104E093A004B2
:1053E0000E941B27219799F7DF91CF911F910F9171
:1053F000FF90EF90DF90CF900895CF93DF93EC0173
:105400008991882319F00E941B27FACFDF91CF9151
:105410000895CF92DF92EF92FF921F93CF93DF9385
:10542000EC016A017B01122F0E94FD29FE0101900F
:105430000020E9F731978E2F8C1BC82FC43128F438
:1054400080E20E941B27CF5FF9CF112331F1C114F5
:1054500084E0D806E104F10400F1C701B6012AE0B6
:1054600096958795779567952A95D1F70E94C029DB
:105470008DEB91E00E94FD29C701B6010E94C02971
:1054800083EC91E00E94FD29DF91CF911F91FF9065
:10549000EF90DF90CF900C944A27C701B6010E948D
:1054A000C029112389F385EC91E0ECCFCF93DF93F2
:1054B000EC010E94D6506EE270E0CE010E94C25014
:1054C000892B39F46CEC71E0CE01DF91CF910C9413
:1054D000B750DF91CF910895CF92DF92EF92FF9274
:1054E0000F931F93CF93DF93C1E0D0E00E94FF1F83
:1054F000A0919204B09193048C91843209F047C03A
:105500001196D12CC12C2A2F9B2F8D9130ED380F65
:105510003A3060F454E0CC0CDD1C5A95E1F7082ECB
:10552000000C990BC097C80ED91EEDCF3FEB380F7A
:10553000363050F444E0CC0CDD1C4A95E1F7082EDF
:10554000000C990BC797EFCF3FE9380F3630A0F02A
:105550002093920490939304CC9DC001CD9D900D17
:10556000DC9D900D1124DF91CF911F910F91FF9041
:10557000EF90DF90CF90089534E0CC0CDD1C3A958D
:10558000E1F7082E000C990B87559109CCCF8D328D
:1055900049F41196B0939304A0939204D195C195C8
:1055A000D109A4CF803341F41196B0939304A09312
:1055B0009204D12CC12CD0CF9FEC980F9930C8F415
:1055C000D12CC12C2AE02C9DA0012D9D500D112421
:1055D0008D91840F952F911D6C0130E3C31AD10872
:1055E0008C9180538A3078F3B0939304A093920403
:1055F000B3CF9FEB980F9A3108F0CCC011969C91D5
:10560000119791549A3180F090E081549048880F1E
:10561000991F2091322030913320820F931FFC017B
:10562000C080D1801196E0CF81EE91E00E943920B8
:1056300000918804083009F4C4C0E0919204F0910C
:1056400093048081883209F0BCC03196F0939304B2
:10565000E09392040E94612C6C01E0919204F0911D
:1056600093048081893209F0ACC03196F0939304A1
:10567000E0939204083008F08DC0402F50E04C5B5E
:10568000544DFA010C94A1504C2B532B592B772BD2
:10569000A02BB22BCA2BBD2BF601EE55FB4F808100
:1056A000C82ED12C59CFD7FE57CFD194C194D10851
:1056B00053CF18E11C0D60E0812F0E94E8081830DC
:1056C00020F0173108F417E1185117701064109387
:1056D0007C0080917A00806480937A0080917A00C7
:1056E00086FDFCCFC0907800D090790035CF60E087
:1056F0008C2D0E94E808B6017727FB01ED54F74F87
:105700008491FB01ED56F74F0491FB01ED58F74FE3
:105710001491112309F44DCF81110E948208E12FC9
:10572000F0E0EE0FFF1FE457FF4FA591B491EC910D
:105730000E2391E080E009F490E0C92ED82E0CCF22
:105740000D2C000CEE08FF08C114D104E104F10493
:1057500009F402CF0E94034BA70196010E94184E44
:105760006B01FACEB601DD0C880B990B0E94254F18
:105770000E9424500E94ED4EF3CFF0E2CF16D104E8
:1057800008F017CFF601EE0FFF1FE15CFB4FC08062
:10579000D180E2CEE0919204F0919304808188322E
:1057A00081F43196F0939304E09392040E94612C6B
:1057B0006C01A0919204B09193048C91893209F408
:1057C00031CF81E080938704F4CE1F93CF93DF9392
:1057D0000E946C2AEC010E94FF1F11E0E0919204EC
:1057E000F091930480818A3281F43196F09393048E
:1057F000E09392040E946C2A9E01289FE001299F59
:10580000D00D389FD00D1124E9CF8F3279F4319625
:10581000F0939304E09392040E946C2ABC01892BBC
:10582000B1F0CE010E948D50EB01D8CF853291F4BA
:105830003196F0939304E09392040E946C2ABC0189
:10584000892B29F0CE010E948D50EC01C7CF109317
:105850008704C4CFCE01DF91CF911F910895CF93DC
:10586000DF93E0919204F091930480818D32B1F046
:105870008B32A1F00E94E52BEC01E0919204F091B3
:10588000930480818D3269F43196F0939304E09310
:1058900092040E94E52BC81BD90BEFCFD0E0C0E0EB
:1058A000ECCF8B3251F43196F0939304E093920451
:1058B0000E94E52BC80FD91FE0CFCE01DF91CF9119
:1058C0000895CF93DF930E942F2CEC0180918704E1
:1058D000811129C086E990E00E943920E091880476
:1058E000E73009F1E73008F042C0F0E0E658F34D48
:1058F0000C94A150812C8A2C972C9F2CA72CAF2C78
:105900008A2C0E942F2C31E020E0C817D9074CF4D4
:1059100030E007C00E942F2C31E020E0C817D907E3
:10592000B9F3C32FD22FCE01DF91CF9108950E94FA
:105930002F2C31E020E08C179D079CF3E9CF0E94CB
:105940002F2C31E020E0C817D90711F7EACF0E94C9
:105950002F2C31E020E08C179D071CF7D9CF0E9437
:105960002F2C31E020E0C817D907DCF2D1CFD0E0EE
:10597000C0E0D9CF2F923F924F925F926F927F9269
:105980008F929F92AF92BF92CF92DF92EF92FF924F
:105990000F931F93CF93DF93CDB7DEB7C05DD109CF
:1059A0000FB6F894DEBF0FBECDBF0E94241F1E01AC
:1059B00021E4220E311CA101485F5F4FC753DF4F26
:1059C00059834883C95CD0408CE993E29C0150E044
:1059D00040E0C553DF4F288339834A835B83CB5C28
:1059E000D040AE01425A5F4FC254DF4F59834883C3
:1059F000CE5BD0408BE790E08C0F9D1F0C96C1537F
:105A0000DF4F99838883CF5CD04081E0809334203E
:105A10001092900410928F048091220190912301A2
:105A20008E559B4F9093A1048093A00486EB93E046
:105A30000E9467270DC0F0938004E0937F04E5CFB8
:105A4000B0933120A09330201093930400939204DC
:105A500080919B04813031F510929B040E94FF1FBE
:105A6000E0919204F091930480818A3011F00C94BB
:105A7000013A10928E0410928D040E94E51F9093BB
:105A80008C0480938B0420918B0430918C04809142
:105A90003020909131202817390709F4B6CF0E94A1
:105AA0000729F1CF8230E1F410929B048091811F8D
:105AB0009091821F9093900480938F0480918F0423
:105AC00090919004209130203091312082179307DB
:105AD00009F49BCF03969093930480939204E2C0C1
:105AE00081E08093342080919404882319F01092EF
:105AF0009404DCCF0E9423280E94C61FE09030202F
:105B0000F090312087010E5F1F4FD801FD013196C3
:105B10008C918A30E1F5B0939304A0939204209184
:105B2000322030913320BF01C901FB014291BF01F6
:105B3000FC014293CF0106171707B9F7C8018A1B6A
:105B40009B0B0197820F931F909393048093920471
:105B50000E940F206C0190938E0480938D040E940C
:105B6000FF1FC114D10409F494C0FFEFCF16DF0664
:105B700009F47FC0A0909204B090930480E0F501F6
:105B8000E80FF11D90819A3021F08F5FF8CFDF018F
:105B9000BDCFA4E09A2E980E8501035011091093F1
:105BA000930400939204D801CD92DC92F5013197D1
:105BB00090820E94E51FFC01E816F906D1F0808171
:105BC0009181C816D906A9F482819F01280F311D41
:105BD000E81AF108AF014E155F0539F0D9018D9132
:105BE0009D01DA018D93AD01F6CF509331204093A2
:105BF0003020D5018C918A3009F42ACFA091302031
:105C0000B0913120992009F41BCF98012A1B3B0B3E
:105C1000892D90E02817390708F4C9019D01280F44
:105C2000391FA9016D01662777276E1B7F0B76014F
:105C3000E60EF71EEF2861F4D801AF01480F591F97
:105C4000E417F50761F4981A080F191FD901DACF84
:105C5000D601FE906D01DA01FE92AD01E8CF6D91A3
:105C60006193EECFF0938004E0937F048EE993E09C
:105C7000DFCE89E893E0DCCE87E693E00E946727D9
:105C8000C4CE0E947B1E80938620882309F485C0A1
:105C90007EC01093930400939204F70182818A30AE
:105CA00009F4D6CE80918620882339F00E94D31E35
:105CB0004B9749F480E693E0E1CF0E947B1E8093EE
:105CC00086208111F3CF85E592E00E943920109162
:105CD0008804113408F078C0E12FF0E0EE58F14D5F
:105CE0000C94A1502E2DF02E082FCB386F39112F88
:105CF000252F9638E838E42EFA379937683A3C2F42
:105D00004A2F243B2E3CAC3C053DE42E5A3D783EC8
:105D1000683AE42E013F313FB32E3C2FAF3FBE2EF9
:105D2000C63F3B40DA40C9418243DA43464481449E
:105D3000922F3D30BB2F1B3053307D30DC3000358F
:105D4000FB3378340E365C3675368C360537603169
:105D500004328931E431193243328832F83EB63E9A
:105D6000823E873E6F39109287040E94612CBC01ED
:105D7000990F880B990B0E943E0926C00E94D706F6
:105D800010922C2080918620882309F47ACF0E94DB
:105D9000D31E90938A0480938904809192049091F9
:105DA0009304FC01019620812A33D9F3F0939304E4
:105DB000E09392040E94FF1FE0919204F0919304FB
:105DC00080818A3009F06ECFE0918F04F0919004C9
:105DD000309709F43DCE82818E0F9F2F911D6ACEA0
:105DE000E0919204F091930480818A3011F00C9438
:105DF00000408DE793E20E94CF25109229208091E8
:105E0000811F9091821F909331208093302020CE6B
:105E100010928604109285041092840410928304D8
:105E200045CE109287040E94612C20918704211195
:105E30001DCFE0919204F091930420812A3009F45F
:105E400015CF892B09F02ECFBFCF109287040E9467
:105E5000612C90938E0480938D048091870481112E
:105E600005CFE0919204F091930480818A3009F08B
:105E7000FDCE0E94E51F1ECEE0919204F0919304A6
:105E800080818A3011F00C940040809130209091F4
:105E9000312010CE0E94D70610922F2010E11093CF
:105EA0002C2085ED94E00E946727C0903220D0908E
:105EB00033208091302090913120C81AD90A0D2CBE
:105EC000000CEE08FF0881ED91E00E94FD2980E2C0
:105ED0000E941B27C701B6010E94C0298AED91E0EC
:105EE0000E94FD290E944A2710922F2010932C20F7
:105EF000C053DF4F0FB6F894DEBF0FBECDBFDF91AA
:105F0000CF911F910F91FF90EF90DF90CF90BF90B6
:105F1000AF909F908F907F906F905F904F903F9049
:105F20002F90089510E000E0C8010E941927282F43
:105F300030E02115310509F447CF2A30310529F425
:105F400090912C20985F90932C20A90140525109E8
:105F50004F35510538F02A30310521F02D3031050B
:105F600009F08FE30E941B270F5F1F4F0115F0E11F
:105F70001F07D1F629CF8CEE91E00E943C068DE000
:105F80000E94EA058AE00E94EA05812C912C5401C6
:105F900010E000E0F8E2EF2EF12C60E0C8010E9472
:105FA0000A4EC801B7010E947950892BB9F480913B
:105FB0002C2078E0D72ED80E10927120D09272202B
:105FC000C501B401ECE09695879577956795EA95BC
:105FD000D1F70E9475208D2D0E946E08C8018F7721
:105FE0009927892B19F48EE20E941B270F5F1F4F00
:105FF00024E6820E911CA11CB11C811430E493068E
:1060000036E0A306B10449F610912C20185F1092D7
:1060100071201093722064E670E080E090E00E94AE
:106020007520812F0E946E080E944A2780E592E029
:106030000E946727C9CE10922C200E94D70681E0CB
:1060400080932A2010929D0410929C040E94E51FC8
:1060500090938C0480938B0420918B0430918C045A
:1060600080913020909131202817390719F00E9433
:106070000729F2CF10922A20C8CC10922C200E941F
:10608000D7068091811F9091821F90933120809339
:10609000302010929D0410929C0481E0809328206F
:1060A00080932920B2CC109287040E94612C182F73
:1060B0008091870481110C9400400E94FF1FE091A1
:1060C0009204F091930480818C3211F00C94004082
:1060D0003196F0939304E09392040E94FF1F109274
:1060E00087040E94612C9091870491110C940040C8
:1060F000612F90E00E940A4E45CE0E94FF1FE09162
:106100009204F091930400818FEB800F8A3190F517
:1061100010E001541048000F111F8091322090911F
:106120003320080F191F3196F0939304E0939204E3
:106130000E94FF1FE0919204F091930480818C32C1
:1061400011F00C9400403196F0939304E093920484
:106150000E94FF1F109287040E94612C20918704E7
:1061600021110C9400400E94192790E0D8018D93D2
:106170009C9308CE109287040E94612C2091870482
:1061800021110C9400400E941927182F8EEF91E0E6
:106190000E94FD29612F70E090E080E00E94C029FC
:1061A0000E944A2784E092E00E94FD29812F0E94EC
:1061B00031290E944A27E6CD10922C200E94D70652
:1061C0000E94FF1FE0919204F09193048081C12C02
:1061D000D12C7601882319F00E940F206C010E94B7
:1061E0004A2786010219130950E1C52ED12CC1019D
:1061F000800F911F0E9468298AE30E941B2780E27A
:106200000E941B277101C8018E0D9F1D0E94192736
:10621000B82E81E1ECEAF1E0DE01119601900D92D9
:106220008A95E1F7EB2DE295EF7021E030E02C0F3D
:106230003D1F2E0F311DF901AB2DAF7041E050E035
:106240004C0F5D1F4A0F511DDA01AC9080810E94F6
:106250001B278A2D0E941B2780E20E941B2780EEAD
:106260008B0D8F3548F5D701BC923FEFE31AF30A47
:10627000C753DF4F48815981C95CD0404E155F0537
:1062800011F6D10150961C928CE70E941B275101F8
:10629000F50181915F010E941B27EA14FB04C1F7FD
:1062A0000E944A27F1E0CF1AD108085F1F4FC1149E
:1062B000D10409F09CCF88CD2EE2F7012083D5CF01
:1062C00010E000E0C8010E942C22282F30E02F3F70
:1062D000310509F479CD2A30310529F490912C202B
:1062E000985F90932C20A901405251094F355105D8
:1062F00038F02A30310521F02D30310509F08FE3D7
:106300000E941B270F5F1F4F013020E21207D1F6BA
:106310005BCD8AE092E00E943C068DE00E94EA0597
:106320008AE00E94EA05812C912C540110E000E0E3
:1063300041E5E42EF12C6FEFC8010E94FC1EC8015C
:10634000B7010E947950892BB9F480912C2028E064
:10635000D22ED80E10927120D0927220C501B401B5
:106360003DE096958795779567953A95D1F70E9488
:1063700075208D2D0E946E08011103C08EE20E94CF
:106380001B270F5F1F4F34E6830E911CA11CB11C0D
:10639000811440E894064CE0A406B10461F6109123
:1063A0002C20185F109271201093722064E670E028
:1063B00080E090E00E947520812F0E946E080E946C
:1063C0004A278BE492E034CE10922C200E94D7060C
:1063D00083E080932A2010929D0410929C040E94D6
:1063E000E51F90938C0480938B0420918B04309153
:1063F0008C0480913020909131202817390709F4BE
:1064000039CE0E940729F1CF10922C200E94D70686
:106410008091811F9091821F909331208093302032
:1064200010929D0410929C0481E08093282083E0C8
:1064300037CE109287040E94612C182F8091870418
:1064400081110C9400400E94FF1FE0919204F09192
:10645000930480818C3211F00C9400403196F093BB
:106460009304E09392040E94FF1F109287040E94FD
:10647000612C9091870491110C940040612F90E061
:106480000E94FC1E7FCC0E94FF1FE0919204F091BD
:10649000930400818FEB800F8A3170F510E0015476
:1064A0001048000F111F8091322090913320080F67
:1064B000191F3196F0939304E09392040E94FF1FFA
:1064C000E0919204F091930480818C3211F00C944D
:1064D00000403196F0939304E09392040E94FF1FD2
:1064E000109287040E94612C2091870421110C9442
:1064F00000400E942C2239CE109287040E94612C09
:106500002091870421110C9400400E942C223DCE42
:1065100010922C200E94D7060E94FF1FE091920447
:10652000F09193048081C12CD12C7601882319F03D
:106530000E940F206C010E944A278601021913094C
:1065400080E1C82ED12CC101800F911F0E946829C3
:106550008AE30E941B2780E20E941B277101C7016A
:10656000800F911F0E942C22B82E81E1ECEAF1E00D
:10657000DE01119601900D928A95E1F7EB2DE295DF
:10658000EF7021E030E02C0F3D1F2E0F311DF9017F
:10659000AB2DAF7041E050E04C0F5D1F4A0F511D15
:1065A000DA01AC9080810E941B278A2D0E941B2754
:1065B00080E20E941B2780EE8B0D8F3548F5D701B6
:1065C000BC923FEFE31AF30AC753DF4F488159816A
:1065D000C95CD0404E155F0511F6D10150961C9252
:1065E0008CE70E941B275101F50181915F010E94F8
:1065F0001B27AE14BF04C1F70E944A27F1E0CF1A4F
:10660000D108085F1F4FC114D10409F09CCFDCCB27
:106610002EE2F7012083D5CFEF961FAE1EAEEF9787
:10662000C158DF4F488259826A827B82CF57D0405F
:106630004CE951E0ED965FAF4EAFED97CC56DF4F92
:1066400019821882C459D040C957DF4F1882C758E1
:10665000D04096C2EF961FAE1EAEEF97C158DF4FE7
:10666000488259826A827B82CF57D0408CE991E080
:10667000ED969FAF8EAFED97E1CFD3948389948948
:10668000A589B689880E991EAA1EBB1E6EE270E00F
:106690008BE294E00E94C2508C01009709F46CC018
:1066A0009C012B5234407901A9016BE274E082E233
:1066B00094E00E94DD50F701EE5DFB4F1082B801BF
:1066C0006F5F7F4F43E050E08EE194E00E94DD5029
:1066D000109221048FEC90E00E94582782E294E00F
:1066E0000E943C06E2E2F4E001900020E9F70CE2AF
:1066F00014E00E1B1F0B1016110614F001E010E041
:10670000F12CE12C89EF90E00E9458273FEFE31A2B
:10671000F30AE016F106B4F38EE194E00E943C0621
:10672000EEE1F4E001900020E9F709E214E00E1B2D
:106730001F0B1016110614F001E010E0F12CE12CF3
:1067400089EF90E00E9458274FEFE41AF40AE01610
:10675000F106B4F3CC56DF4FE881F981C459D0403B
:1067600080E090E0DC01309721F083899489A5894D
:10677000B6890E94A8284AC248E050E06BE274E063
:1067800082E294E00E94DD5083E0EDECF1E0AEE1C6
:10679000B4E001900D928A95E1F710922A049ACF05
:1067A000CE018A569F4F0E94CF250E944A2786EC31
:1067B00090E00E9458278D2D90E00E94A8288AEB37
:1067C00090E00E945827C4010E94A82883EB90E023
:1067D0000E9458270E944A278AEA90E00E94582780
:1067E0008C2D90E00E94A82882EA90E00E94582711
:1067F0000E944A270AC910928604109285041092BA
:1068000084041092830480E492E00E9467278091C0
:10681000811F9091821F909331208093302010929D
:1068200087040E945F1F2091870421110C9400406F
:10683000BC01CE01825A9F4F0E94562A6AEA71E03B
:1068400080E091E00E94CD508E010F5F1F4F892B99
:1068500011F5C154DF4F5881CF5BD0405F93C254D4
:10686000DF4F8881CE5BD0408F9383E392E09F938C
:106870008F931F930F930E94F7500F900F900F90DC
:106880000F900F900F90C8010E944A24811121C0DF
:1068900081E392E0F3C9C154DF4F9881CF5BD040D0
:1068A0009F93C254DF4FA881CE5BD040AF9380E06E
:1068B00091E09F938F9381E392E09F938F931F9337
:1068C0000F930E94F7500FB6F894DEBF0FBECDBFF6
:1068D000DACF41E0B801C1010E941626C1010E9431
:1068E000480684E08093292081E0809328208DC889
:1068F00087E292E00E946727109287040E945F1F40
:106900002091870421110C940040BC01CE01825AD1
:106910009F4F0E94562A6AEA71E080E091E00E944F
:10692000CD508E010F5F1F4F892B09F043C0C1541A
:10693000DF4FF881CF5BD040FF93C254DF4F2881F7
:10694000CE5BD0402F9383E392E09F938F931F936E
:106950000F930E94F7500F900F900F900F900F9091
:106960000F90C8010E944A24882329F06DED74E23B
:10697000C8010E94992347E1B801C1010E9416266F
:10698000C1010E94480684E080932A200E94E51FEE
:1069900090938C0480938B0420918B0430918C0411
:1069A00080913020909131202817390709F10E94F9
:1069B0000729F2CFC154DF4F3881CF5BD0403F93DE
:1069C000C254DF4F4881CE5BD0404F9380E091E0CE
:1069D0009F938F9381E392E09F938F931F930F93E5
:1069E0000E94F7500FB6F894DEBF0FBECDBFB9CFEF
:1069F00010922A208DE793E20E94CF250E94D706AD
:106A00000E94D70610922C2089ED90E00E94672703
:106A10000E944A2780E292E00E943C0680E091E0DA
:106A20000E943C060E944A270E944A2741E060E0FB
:106A300071E0CE018A569F4F0E941626C155DF4F46
:106A400088819981CF5AD040009729F040E050E0EA
:106A5000BA010E94F114C12CD12C812C912C54012B
:106A6000B8EE4B2EB3E05B2E612C712CC155DF4F7D
:106A700008811981CF5AD040D80115968C9115976D
:106A8000823008F4E7CD1A968D919D910D90BC91BE
:106A9000A02D8F719927AA27BB27892B8A2B8B2B97
:106AA00009F0D8CD40E250E0BE016F5F7F4FC801D2
:106AB0000E948516803209F0CDCD8981882309F4A2
:106AC000C9CD853E79F38E3269F38C8583FDEACF9B
:106AD000A2961FAE1EAEA297E0E9F1E0A096FFAF2E
:106AE000EEAFA097A4961FAEA497BE016F5F7F4F35
:106AF000E0E080E0DB019D91BD019032A9F088309B
:106B000051F421EB30E02C0F3D1F2E0F311DFEE222
:106B1000D901FC93EF5F21EB30E02C0F3D1F2E0FCE
:106B2000311DD9019C93EF5F8F5F8B3019F721EBFB
:106B300030E02C0F3D1F2E0F311DF9011082C15581
:106B4000DF4F68817981CF5AD04021E0AE014F54A8
:106B50005F4FCE01825A9F4F0E948F22882309F4F3
:106B60005BCDBE01625A7F4FC1010E945A1AAE012D
:106B70004F545F4FB101CE0185589F4F0E94E125D0
:106B8000CC56DF4F08811981C459D0400115110539
:106B900009F406CED80115968C91882309F400CE0D
:106BA000C153DF4F68817981CF5CD0408BE294E0A4
:106BB0000E94D650F8018581823008F45ECDC394DE
:106BC00087ED90E00E9458278BE294E00E943C06FB
:106BD000EBE2F4E001900020E9F70FE314E00E1B74
:106BE0001F0B1016110614F001E010E0F12CE12C3F
:106BF00089EF90E00E945827FFEFEF1AFF0AE01696
:106C0000F106B4F381ED90E00E9458270E944A27D4
:106C1000CE0185589F4F0E94CF2528CF10922C205F
:106C20000E94D706109287040E945F1F209187045C
:106C300021110C940040BC01C1010E94562A6AEA4D
:106C400071E080E091E00E94CD508E010F5F1F4FF8
:106C5000892BF1F43F922F9283E392E09F938F93DD
:106C60001F930F930E94F7500F900F900F900F906B
:106C70000F900F90C8010E944A246DED74E28111BB
:106C800030C010922A208DE793E20E94CF25B8CE23
:106C90003F922F9280E091E09F938F9381E392E067
:106CA0009F938F931F930F930E94F7500FB6F89402
:106CB000DEBF0FBECDBFDECF10922C200E94D706C4
:106CC000109287040E945F1F8C01809187048111BC
:106CD0000C940040C8010E944A248111D2CF6DE07B
:106CE00075E2C8010E949923CCCF10922C200E94FB
:106CF000D706109287040E945F1F8C018091870441
:106D000081110C940040C8010E944A246BE774E290
:106D1000882309F4B6CFE5CF10922C200E945F1F84
:106D2000F82EE92E67E372E00E94CD50892B39F4EA
:106D30006AEA71E080E091E00E94D65061CE69E39A
:106D400072E08F2D9E2D0E94CD50892B79F46FE239
:106D500070E080E091E00E94EC50009749F3B1E0D0
:106D600080309B0729F3FC0110824ACE6AEA71E069
:106D700080E091E00E94CD508E010F5F1F4F892B64
:106D800019F5EF92FF9283E392E09F938F931F9305
:106D90000F930E94F7500F900F900F900F900F904D
:106DA0000F9041E0B801C1010E941626D101599609
:106DB000ED91FC91309719F08581811119C083E123
:106DC00092E00E9467271CCEEF92FF9280E091E054
:106DD0009F938F9381E392E09F938F931F930F93E1
:106DE0000E94F7500FB6F894DEBF0FBECDBFD9CFCB
:106DF000823028F0C1010E94CF25B8019BCF83E0EB
:106E000092E00E946727C10140CF0E94D7061092EE
:106E10002C208CE392E00E943C0680913F2382303C
:106E200009F47EC0833009F47EC0813009F07EC051
:106E300083E492E00E943C068CE592E00E943C06CE
:106E40006091572370E090E080E00E94C0290E948A
:106E50004A270E944A2782E792E00E943C066091FE
:106E6000492370914A2380914B2390914C230E9497
:106E7000C0290E944A278DE792E00E943C0660915B
:106E8000442370E090E080E00E94C0290E944A27DD
:106E900080E992E00E943C06A0914423209149237E
:106EA00030914A2340914B2350914C23B0E00E94F3
:106EB000374E0E94C029A09144232091492330914C
:106EC0004A2340914B2350914C23B0E00E94374E0F
:106ED0006B017C010E944A270E944A278FE992E0B9
:106EE0000E943C06C701B6019695879577956795F0
:106EF0000E94C0290E944A2782EB92E00E943C0631
:106F0000C701B601ABE09695879577956795AA95E9
:106F1000D1F70E94C0290E944A270E944A2768CCC4
:106F200089E492E087CF8FE492E084CF84E592E019
:106F300081CFB1E0B09334200E94FF1FE091920412
:106F4000F091930410818FEB810F8A3110F00C9433
:106F5000362E3196F0939304E09392040E94FF1F23
:106F6000E0919204F091930480818A3021F08A3379
:106F700011F00C94004080919204909193049093AE
:106F8000820480938104109291040E9423288091AE
:106F9000910481110C945A2E0E94C61F80913020BA
:106FA00090913120029690939304809392040E94D2
:106FB000FF1F109287040E94612C209187042111E9
:106FC000DACF212F30E021543048220F331F409177
:106FD000322050913320240F351FF9019183808393
:106FE0008091810490918204909393048093920401
:106FF0000C94C22E0E94FF1FE0919204F091930422
:10700000B0808FEB8B0D8A3110F00C9400403196DC
:10701000F0939304E09392040E94FF1FE091920486
:10702000F091930480818D3311F00C9400403196DF
:10703000F0939304E09392040E94FF1F1092870440
:107040000E94612C7C018091870481110C94362E62
:1070500080E092E00E943920809188048111D0C79D
:107060000E94612C8C018091870481110C94362E32
:107070008BEF91E00E94392080918804811152C0E9
:107080000E94612C6C018091870481110C94362E32
:107090000E94FF1F4091920450919304DA018C9159
:1070A0008A3019F08A3309F0ABC7909187049111A7
:1070B0000C94362E8A3011F00C94362EE091A004F8
:1070C000F091A104CF010A9620919E0430919F0473
:1070D0008217930710F40C943C2E3A97F093A10476
:1070E000E093A0048B2D90E081549048880F991F65
:1070F0002091322030913320820F931FDC01ED92DA
:10710000FC92B6E4B083B18213830283D582C48239
:107110005187408780918F04909190049783868354
:107120000C94C22ECC24C394D12CB2CF10928704DD
:107130000E94612C90938E0480938D04809187042B
:1071400081110C94362EA0919204B09193048C91ED
:107150008A3009F055C7E091A004F091A104CF0155
:10716000059620919E0430919F048217930710F496
:107170000C943C2E3597F093A104E093A00487E48F
:107180008083B483A38380918F0490919004928331
:1071900081830C94392F0E94FF1FE0919204F0919B
:1071A0009304808181548A3110F00C94362E3196EC
:1071B000F0939304E09392040E94FF1FE0919204E5
:1071C000F091930480818A3319F08A3009F018C74E
:1071D0002091A0043091A1043093800420937F0477
:1071E00040912201509123014F555B4FA091920491
:1071F000B0919304F9011197E417F50710F00C947E
:10720000322E8081863401F1873411F00C941B2DCD
:107210001830C1F4F0938004E0937F04818192815F
:107220009093900480938F0483819481909393042E
:10723000809392042B5F3F4F3093A1042093A004CE
:107240000C94C22E3596D8CF133009F046C08C91DD
:1072500090E06181062E000C770B86179707E9F501
:10726000F0938004E0937F0481549048880F991F25
:10727000A0913220B0913320A80FB91F2D913C91DD
:10728000119784819581280F391F2D933C93848118
:1072900095811816190664F48281938182179307E9
:1072A00074F43A96F093A104E093A0040C94C22ED7
:1072B000892BB9F3828193812817390794F380854C
:1072C0009185909393048093920486819781909303
:1072D000900480938F040C94C22E3A968DCFE09147
:1072E0009204F09193040081013409F04AC0818135
:1072F000823509F046C08281883209F042C0339657
:10730000F0939304E0939204109287040E94612CFE
:107310008C018091870481110C94362EE0919204A7
:10732000F09193048081893209F06AC63196F09316
:107330009304E09392040E94FF1FE0919204F09165
:10734000930480818D3309F05BC63196F0939304EA
:10735000E09392040E94FF1F0E94612C20918704F9
:1073600021110C94362E0032110510F00C94362E9B
:10737000000F111FF801E15CFB4F918380830C9497
:10738000C22E8FEB800F8A3110F00C94362E10E055
:1073900001541048000F111F80913220909133202A
:1073A000080F191F3196F0939304E09392040E9402
:1073B000FF1FE0919204F091930480818D3309F0D6
:1073C0001FC63196F0939304E09392040E94FF1F2E
:1073D000109287040E94612C9C0180918704811186
:1073E0000C94362EE0919204F091930490819A309F
:1073F00019F09A3309F004C6F801318320830C9404
:10740000C22E109287040E94612C8C018091870407
:107410008111F6C50E94FF1FE0919204F091930440
:1074200080818A30B9F410938E0400938D040E94F9
:10743000E51F90938C0480938B0420913020309131
:1074400031208217930711F40C94052D0E9407290F
:107450000C94052D8C3209F0D3C53196F09393042A
:10746000E09392040E94FF1F109287040E94612CF7
:107470007C01809187048111C3C5E0919204F09151
:10748000930480818A3009F0BBC510938E04009369
:107490008D040E94E51F90938C0480938B0410E070
:1074A00000E00E151F0511F40C94052D20918B049E
:1074B00030918C0480913020909131202817390729
:1074C00011F40C94052D0E9407290F5F1F4FE9CF7F
:1074D00010923420E0919204F091930480818A33D9
:1074E00041F40E944A27809192049091930401965E
:1074F0007BCD8A3011F40C94E42E0E94FF1FE091A2
:107500009204F09193041081123211F0173259F461
:107510003196F0939304E09392048191181709F443
:107520003FC08A30D1F70091920410919304D801A2
:107530008C91823209F464C5873209F461C581EE09
:1075400091E00E94392080918804863009F052C071
:107550000E94FF1FE0919204F09193048081883291
:1075600009F04EC53196F0939304E0939204109283
:1075700087040E94612C9091870491110C94362EFF
:10758000E0919204F09193049081993209F038C50A
:107590003196F0939304E09392040E94EA051DC093
:1075A000E0919204F09193048081181789F00E9471
:1075B0001B278091920490919304019690939304D9
:1075C0008093920480912F208A5F80932F20E8CFB0
:1075D0003196F0939304E0939204E0919204F09139
:1075E000930480818C32B1F43196F0939304E0934C
:1075F000920483CF10939304009392041092870413
:107600000E94612C2091870421110C94362E0E9437
:10761000CF28E3CF8B3381F481818A3019F08A330C
:1076200009F0EEC43196F0939304E0939204B1E034
:10763000B09334200C94C22E8A3019F08A3309F0AA
:10764000DFC40E944A27F3CF0E94D70610922C2055
:1076500080ED91E00E9467278BEA91E00E94672706
:1076600040913020509131208091811F9091821F54
:10767000481B590B052E000C660B770B21E085EC9F
:1076800092E00E94092A409122015091230170E06A
:1076900060E021E084ED92E00E94092A40919E047E
:1076A00050919F0470E060E020E083EE92E00E9441
:1076B000092A21E046E350E060E070E08FEE92E0BE
:1076C0000E94092A21E042E350E060E070E089EF87
:1076D00092E00E94092A4091A0045091A10470E018
:1076E00060E020E089E093E00E94092A21E0C55390
:1076F000DF4F488159816A817B81CB5CD0408DE02E
:1077000093E00E94092A40913220509133208091C9
:10771000302090913120481B590B052E000C660B30
:10772000770B21E08AE193E00E94092A8091982357
:1077300090919923009711F48CE993E2AE014F5F89
:107740005F4F481B590B052E000C660B770B21E091
:1077500085E293E00E94092A0E944A270E944A2754
:1077600080EA91E00E9467278BE791E00E946727FB
:107770008FE293E00E943C068091811F9091821FCE
:107780000E949A1F85EC93E00E943C060E944A27C3
:1077900084E493E00E943C06809130209091312057
:1077A0000E949A1F85EC93E00E943C060E944A27A3
:1077B00089E593E00E943C0680913220909133202D
:1077C0000E949A1F85EC93E00E943C060E944A2783
:1077D0008EE693E00E943C0680919E0490919F0467
:1077E0000E949A1F85EC93E00E943C060E944A2763
:1077F00083E893E00E943C068091A0049091A1044C
:107800000E949A1F85EC93E00E943C060E944A2742
:1078100088E993E00E943C068CE993E20E949A1F5B
:1078200085EC93E00E943C060E944A278DEA93E093
:107830000E943C060E944A270E944A270E944A272B
:10784000109296040E9471096093970470939804B3
:107850008093990490939A040C94052D0E94D70666
:1078600010922C2010E000E0C8010E9419270F5F41
:107870001F4F0115E0E11E0711F08111F5CF0150F6
:1078800011096801110FEE08FF088CE691E00E94D3
:10789000672787E491E00E94672721E040E050E1FC
:1078A00060E070E087EC93E00E94092A21E0B701D4
:1078B000A60182ED93E00E94092A40E050E160E0D9
:1078C00070E04C195D096E097F0921E08CED93E0B1
:1078D0000E94092A0E944A270E944A2788E391E0D1
:1078E0000E94672783E191E00E94672710E000E093
:1078F000C8010E942C228F3F31F00F5F1F4F0115EE
:10790000F0E21F07A9F71016110614F001E010E0CD
:10791000015011096801110FEE08FF0821E040E055
:1079200050E260E070E087EC93E00E94092A21E0D9
:10793000B701A60182ED93E00E94092A40E050E2DF
:1079400060E070E04C195D096E097F0921E08CED63
:1079500093E00E94092A70CF0E94D70610922C2033
:10796000E0919204F091930480818A3029F586EEAB
:1079700093E00E943C06609122017091230190E007
:1079800080E00E94C0290E944A2782EF93E00E9473
:107990003C0668EE73E080E090E00E94C0290E94FF
:1079A0004A2788EF93E00E943C066CE47DE180E08A
:1079B00090E00E94C02942C30E94612C209187045C
:1079C00021111EC38C018D349D4114F00CE41DE186
:1079D000083E33E0130714F408EE13E0109323017C
:1079E000009322018091811F9091821F90933120FA
:1079F000809330200E94241F8EEF93E00E943C066B
:107A0000B801110F880B990BD4CF109287040E94F4
:107A1000612C8C018091870481110C94362EE091A9
:107A20009204F091930480818C3209F0E9C231967E
:107A3000F0939304E09392040E94612C20918704B8
:107A400021110C94362EE0919204F0919304208140
:107A50002A3009F0D5C2093E43E01407F9F04CF48E
:107A6000083E134099F08BE094E00E943C060C9491
:107A7000D9300A3EB3E01B07B9F00B3E134099F72B
:107A80008093722080932C200C94C22E21E0892BAD
:107A900009F420E0209334200C94C22E909321010D
:107AA000809320010C94C22E8093712080932F200C
:107AB0000C94C22EE0919204F091930400818FEB1C
:107AC000800F8A3108F09CC2E0903220F090332081
:107AD00010E001541048000F111F0E0D1F1D3196AC
:107AE000F0939304E09392040E94FF1FE0919204AC
:107AF000F091930480818C3209F06BC03196F09341
:107B00009304E09392040E94FF1FE0919204F0918D
:107B1000930480819FEB980F9A3108F071C290E036
:107B200081549048880F991FE80EF91E3196F09302
:107B30009304E09392048091850490918604892BAC
:107B400061F48091811F9091821F909386048093AD
:107B50008504109284041092830480918304909190
:107B60008404892B09F046C0A0908504B090860457
:107B70008091302090913120A816B90600F5C09070
:107B80009204D0909304C50103969093930480933C
:107B9000920485E592E00E94392080918804833127
:107BA000D9F40E94FF1F80919204909193049093C6
:107BB000840480938304D0929304C09292048091B1
:107BC000830490918404892BA9F487E091E00C94BC
:107BD0003E2EF12CE12CAFCFD0929304C0929204B0
:107BE000D50112968C91A80EB11CB0928604A09279
:107BF0008504BACFC0909204D090930480918304FE
:107C0000909184049093930480939204109287043B
:107C10000E94612C209187042223A9F0E091850421
:107C2000F091860482818E0F9F2F911D9093860480
:107C3000809385041092840410928304D09293045C
:107C4000C09292048ACFF801918380830E94FF1F23
:107C5000E114F104F1F0E0919204F0919304808139
:107C60008C3221F08BEF90E00C943E2E3196F09305
:107C70009304E09392040E94FF1F109287040E94D5
:107C8000612C2091870421110C94362ED7018D93FD
:107C90009C930E94FF1FE0919204F09193048081D5
:107CA0008C32A9F43196F0939304E09392040E94ED
:107CB000FF1F809192049091930490938404809389
:107CC0008304D0929304C09292040C94C22EE0914B
:107CD0008504F091860482818E0F9F2F911D9093D1
:107CE0008604809385041092840410928304E9CF63
:107CF00010928604109285041092840410928304DA
:107D00000C94C22E1092B1005F980C94C22E109267
:107D10003420E0919204F091930480819FEB980FBE
:107D20009A3108F06DC190E081549048880F991FF6
:107D30002091322030913320820F931F9F012F5FBB
:107D40003F4F309393042093920421812A3009F00D
:107D500057C12091890430918A04FC01318320832A
:107D600010928A04109289040C94C22E10928704F7
:107D70000E94612C8C0180918704811141C10E9475
:107D8000FF1FE0919204F091930480818C3209F0FE
:107D900037C13196F0939304E09392040E94FF1F41
:107DA000109287040E94612C6C01990FEE08FF0865
:107DB00080918704811124C10115110541F4B70197
:107DC000A60190E080E00E942A070C94C22EC11404
:107DD000D104E104F10409F495CFB701A601C8016B
:107DE0000E942A07C701B6010E943E090C94C22EC8
:107DF000109234200E946B27F1E0F09334200C9411
:107E0000C22EE12C109287040E94612CF82E8091E2
:107E100087048111F5C00E94FF1FE0919204F09148
:107E2000930480818C3209F0EBC03196F093930477
:107E3000E09392040E94FF1F109287040E94612C1D
:107E40008C01809187048111DBC0EE2069F061E034
:107E50008F2D0E94E808602F8F2D0E94BA080C9485
:107E6000C22EEE24E394CECF28E1F20E61E08F2DF6
:107E70000E94E80861E08F2D0E94E80801151105B5
:107E800011F460E0E9CF0F3F110511F461E0E4CF98
:107E9000EF2DF0E0ED54F74FE491E250EA3008F0B6
:107EA00059C0F0E0EA5AF04C0C94A150603F663F94
:107EB0006C3F773FAA3FAA3F823F8B3F943F9F3F53
:107EC00084B5806884BD07BD0C94C22E84B58062E1
:107ED00084BD08BD0C94C22E809180008068809380
:107EE000800010938900009388000C94C22E80912A
:107EF000800080628093800010938B0000938A0042
:107F00000C94C22E8091B00080688093B0000093E2
:107F1000B3000C94C22E8091B00080628093B000B8
:107F20000093B4000C94C22E8091900080688093DE
:107F3000900010939900009398000C94C22E8091A9
:107F4000900080628093900010939B0000939A00B1
:107F50000C94C22E003811050CF098CF92CF1092DD
:107F600087040E94612C20918704211149C0BC0123
:107F7000990F880B990B611571058105910511F415
:107F80000C94C22E0E94524B0C94C22E1092870465
:107F90000E94612CD82EE82EF92E80918704811141
:107FA0002FC00E94FF1FE0919204F0919304808102
:107FB0008C3231F53196F0939304E09392040E9451
:107FC000FF1F109287040E94612CC82E082F192FC2
:107FD0000E94FF1FE0919204F091930480818C3203
:107FE00089F53196F0939304E09392040E94FF1F69
:107FF000109287040E94612C20918704222321F192
:108000008BE793E00E94582780918F049091900411
:108010000097A1F0E0919204F091930410811A303E
:1080200011F02EE3208390938C0480938B040E94A4
:108030000729E0919204F091930410830E944A274B
:108040000C94282D81E090E020917F20220F220FB8
:10805000220F2E151F04A0F220917E20201711065A
:1080600078F28330910560F6482F6C2D8D2D0E949B
:10807000461C0C94C22E109287040E94612C182F6B
:10808000882E992E809187048111BACF0E94FF1FFC
:10809000E0919204F091930480818C3209F0B0CF8A
:1080A0003196F0939304E09392040E94FF1F109284
:1080B00087040E94612C782EA82EB92E8091870407
:1080C00081119ECF0E94FF1FE0919204F0919304D2
:1080D00080818C3209F094CF3196F0939304E09331
:1080E00092040E94FF1F109287040E94612C682E48
:1080F000C82ED92E80918704811182CF0E94FF1F44
:10810000E0919204F091930480818C3209F078CF51
:108110003196F0939304E09392040E94FF1F109213
:1081200087040E94612C582EE82EF92E8091870436
:10813000811166CF0E94FF1FE0919204F091930499
:1081400080818C3209F05CCF3196F0939304E093F8
:1081500092040E94FF1F109287040E94612CAC01C0
:108160009091870491114CCF20917F20220F220FF4
:10817000220F30E02815390508F442CF60917E20A7
:1081800070E06A157B0508F43BCF2C153D0508F41B
:1081900037CF6E157F0508F433CF4330510508F013
:1081A0002FCF082F252D462D672D812F0E94251DAD
:1081B0000C94C22E109287040E94612C6C01809155
:1081C000870481111DCF0E94FF1FE0919204F0915E
:1081D000930480818C3209F013CF3196F09393048D
:1081E000E09392040E94FF1F109287040E94612C6A
:1081F0007C0180918704811103CF0E94FF1FE091D1
:108200009204F091930480818C3209F0F9CE31967A
:10821000F0939304E09392040E94FF1F109287044E
:108220000E94612C3C01809187048111E9CE0E945B
:10823000FF1FE0919204F091930480818C3209F049
:10824000DFCE3196F0939304E09392040E94FF1FD7
:10825000109287040E94612C5C0180918704811137
:10826000CFCE0E94FF1FE0919204F0919304808191
:108270008C3209F0C5CE3196F0939304E0939204CA
:108280000E94FF1F109287040E94612C582E80913B
:1082900087048111B5CE0E94FF1FE0919204F091F6
:1082A000930480818C3209F0ABCE3196F093930425
:1082B000E09392040E94FF1F109287040E94612C99
:1082C000C054DF4F8883C05CD04080918704811107
:1082D00097CE80917F20880F880F880F90E08C15B3
:1082E0009D0508F48DCE20917E2030E02E153F05AF
:1082F00008F486CE2A153B0508F482CE861597052C
:1083000008F47ECEC054DF4F3881C05CD0403F3F80
:1083100029F14E2C4A2D4E0D5527551F4A01860135
:108320001127C801860D911DCE53DF4F9983888395
:10833000C25CD040481419048CF4C054DF4F28812B
:10834000C05CD040CE53DF4F48815981C25CD040E1
:10835000B801842D0E94561C4394ECCF6C0C052D63
:108360002E2D462D6E2D8C2D0E94251D1E2D1A0D95
:10837000212F4C2D6E2D8C2D0E94251D212F462D39
:108380006E2D862D0E94251D212F462D612F8C2DAF
:108390000DCF109287040E94612C5C0180918704AC
:1083A00081112ECE0E94FF1FE0919204F091930460
:1083B00080818C3209F024CE3196F0939304E093BF
:1083C00092040E94FF1F109287040E94612CE82EE5
:1083D000882E992E80918704811112CE0E94FF1F52
:1083E000E0919204F091930480818C3209F008CEE0
:1083F0003196F0939304E09392040E94FF1F109231
:1084000087040E94612C8C01809187048111F8CD32
:108410000E94FF1FE0919204F091930480818C32BE
:1084200009F0EECD3196F0939304E09392040E940C
:10843000FF1F109287040E94612CF82E8091870400
:108440008111DECD0E94FF1FE0919204F091930410
:1084500080818C3209F0D4CD3196F0939304E0936F
:1084600092040E94FF1F109287040E94612CD82E54
:10847000809187048111C4CD80917F20880F880F5F
:10848000880F8A151B0408F4BBCD80917E2090E0F4
:108490008815990508F4B4CD8017910708F4B0CD7C
:1084A000902EC054DF4FA882C05CD04028015524D4
:1084B00066246394712C6418750890E080E0841938
:1084C0009509DC01AA0FBB1FCA53DF4FB983A883EC
:1084D000C65CD040BFEFDB1659F0B5017727A2018B
:1084E000460F571F641975092D2D8E2D0E94561C9D
:1084F0006E2D600F4F2D8A2D0E94131C6E2D601B58
:108500004F2D8A2D0E94131C4F2D6E2D802F8A0D0A
:108510000E94131C4F2D6E2D8A2D801B0E94131C50
:10852000CE53DF4F1882C25CD04010E000E0F5016E
:10853000FF27CC53DF4FF983E883C45CD040041598
:10854000150514F00C94C22E77FC13C0F1E04F1AFD
:108550005108CA53DF4F28813981C65CD0402E5F55
:108560003F4FCA53DF4F39832883C65CD040620E29
:10857000731E0F5F1F4FC801880F991F0196680E69
:10858000791EC42C3E2D340DC853DF4F3883C85C90
:10859000D0404E2D4419CF53DF4F4883C15CD040AB
:1085A0005FEFD51609F459C09414150401F12D2D6F
:1085B000CC53DF4F88809980C45CD040800E911EE0
:1085C000A401CC53DF4FA880B980C45CD040A01A6E
:1085D000B10AB501832F0E94561C2D2DA401B501AF
:1085E000CF53DF4F8881C15CD0400E94561CCE53D0
:1085F000DF4FA881C25CD0408A2F90E0CE53DF4F7E
:108600000883C25CD0400817190731F1041515051D
:1086100019F12D2DCC53DF4F88809980C45CD04058
:10862000840C951CA401CC53DF4FA880B980C45C96
:10863000D040A418B508B501802F8E0D0E94561C9D
:108640002D2DA401B5018E2DCE53DF4FB881C25C14
:10865000D0408B1B0E94561C9C2C4F2DC853DF4FC3
:108660006881C85CD040C054DF4FB880C05CD04047
:10867000B00E8B2D0E94131C4F2DC853DF4F688105
:10868000C85CD040C054DF4FA880C05CD040A01A66
:108690008A2D0E94131C4F2DCF53DF4F6881C15C80
:1086A000D0408B2D0E94131C4F2DCF53DF4F68817C
:1086B000C15CD0408A2D0E94131CC054DF4FA8809B
:1086C000C05CD040AC0C4F2DBE2CB00E6B2D8A2D53
:1086D0000E94131CC054DF4F8880C05CD0408C18AF
:1086E0004F2D6B2D882D0E94131C4F2DCE2CC01AA0
:1086F0006C2D8A2D0E94131C4F2D6C2D882D0E94ED
:10870000131C1DCF109287040E94612CD82EE82ED6
:10871000F92E80918704811173CC0E94FF1FE09194
:108720009204F091930480818C3209F069CC3196E7
:10873000F0939304E09392040E94FF1F1092870429
:108740000E94612CC82E082F192F80918704811157
:1087500057CC0E94FF1FE0919204F0919304808116
:108760008C3209F04DCC3196F0939304E09392044F
:108770000E94FF1F0E94FF1FE0919204F09193045A
:108780004191F0939304E093920480917F20880FAD
:10879000880F880F8E151F0408F432CC80917E203C
:1087A0008017110608F42CCC6C2D8D2D0E94C60468
:1087B0000C94C22E109287040E94612C8C0180912F
:1087C000870481111DCC0E94FF1FE0919204F0915B
:1087D000930480818C3209F013CC3196F09393048A
:1087E000E09392040E94FF1F109287040E94612C64
:1087F000BC0190918704911103CC30917F20832F8D
:10880000880F880F880F8017110608F4F9CB209184
:108810007E202617170608F4F3CB432F50E0FA0109
:1088200033E0EE0FFF1F3A95E1F70E171F0624F510
:10883000621710F5649F9001659F300D1124E02FA1
:10884000E695E695E6958091842090918520820FAB
:10885000931FE80FF92FF11D208130E0077080E8A9
:1088600090E002C0959587950A95E2F72823392371
:1088700091E0232B09F490E0892F90E00E94CF280B
:1088800089EF90E00E9467270C94C22E1092870413
:108890000E94612C8C01809187048111B1CB0E94D0
:1088A000FF1FE0919204F091930480818C3209F0D3
:1088B000A7CB3196F0939304E09392040E94FF1F9C
:1088C000109287040E94612C20918704211198CB7B
:1088D00020917F20220F220F220F2017110608F46B
:1088E0008FCB20917E202817190608F489CB880F9A
:1088F000880F880F902F990F090F000F0093712098
:10890000BFC8E0919204F091930400818FEB800F37
:108910008A3108F075CB10E001541048000F111F88
:108920008091322090913320080F191FCF010196BA
:10893000909393048093920481818C3209F060CBF0
:108940003296F0939304E0939204109287040E946D
:10895000612C7C018091870481110C94362EE0916A
:108960009204F091930480818C3209F049CB3196C6
:10897000F0939304E09392040E94612C2091870469
:1089800021110C94362EF801208131812E153F05DE
:1089900014F4F182E082D8012D913C911197821755
:1089A000930714F00C94C22E0C94B7301F920F92C0
:1089B0000FB60F9211242F933F938F939F93AF93F2
:1089C000BF938091362090913720A0913820B091AC
:1089D00039203091352023E0230F2D3768F126E828
:1089E000230F0296A11DB11D2093352080933620C0
:1089F00090933720A0933820B093392080913A206B
:108A000090913B20A0913C20B0913D200196A11D6A
:108A1000B11D80933A2090933B20A0933C20B093CB
:108A20003D20BF91AF919F918F913F912F910F90DA
:108A30000FBE0F901F9018950196A11DB11DD4CFA8
:108A40001F920F920FB60F9211240BB60F922F9315
:108A50003F934F935F936F937F938F939F93AF93C6
:108A6000BF93EF93FF9389E892E20E94130EFF9168
:108A7000EF91BF91AF919F918F917F916F915F9196
:108A80004F913F912F910F900BBE0F900FBE0F9003
:108A90001F9018951F920F920FB60F9211240BB6CC
:108AA0000F922F938F939F93EF93FF93E0919922CF
:108AB000F0919A228081E0919F22F091A02282FD84
:108AC0001DC090818091A2228F5F8F732091A3227D
:108AD000821741F0E091A222F0E0E757FD4D958F1B
:108AE0008093A222FF91EF919F918F912F910F90F0
:108AF0000BBE0F900FBE0F901F9018958081F2CF84
:108B00001F920F920FB60F9211240BB60F922F9354
:108B10003F934F935F936F937F938F939F93AF9305
:108B2000BF93EF93FF938091B900887F803609F45B
:108B30004DC008F040C0883209F4A9C028F5803142
:108B400009F49DC0C8F4882309F407C1883009F4EA
:108B500096C0FF91EF91BF91AF919F918F917F91BF
:108B60006F915F914F913F912F910F900BBE0F909E
:108B70000FBE0F901F901895883109F488C080327D
:108B800041F78093482014C0803409F4A5C040F414
:108B90008033B9F38833E9F68093482085ECBCC074
:108BA000803509F489C0883509F49EC0883489F677
:108BB0000E94B90ECECF883909F494C038F58837B1
:108BC00029F050F4883611F0803719F683E080934D
:108BD0004A2010921C2057C0883809F483C080397D
:108BE00019F0803809F0B5CF80911C20803208F050
:108BF00079C0E0911C2081E08E0F80931C20809131
:108C0000BB00F0E0E450F04E80833DC0803B39F083
:108C1000E0F4803A09F485C0883A09F09ACF84E0FC
:108C200080934A201092FB1F1092FA1FE09123209C
:108C3000F091242009958091FA1F81110FC081E0E5
:108C40008093FA1F1092DA1F09C0803C09F4A6CF66
:108C5000883C09F4A3CF883B09F07BCFE091FB1F50
:108C600081E08E0F8093FB1FF0E0E652F04E808192
:108C70008093BB009091FB1F8091FA1F31C08091BF
:108C800043208093BB0085EC8093BC0062CF909121
:108C90004520809144209817B8F580914620909106
:108CA0004720E091452021E02E0F20934520E80F3A
:108CB000F92FF11D8081E5CF20914620309147208A
:108CC000E091452081E08E0F809345208091BB008C
:108CD000E20FF32FF11D8083909145208091442075
:108CE000981788F285E8D0CF209146203091472010
:108CF000E091452081E08E0F809345208091BB005C
:108D0000E20FF32FF11D808380914920811150CF14
:108D100081E08093422084EA8093BC0010924A2034
:108D200018CF85EC8093BC0010924A2080911C20C3
:108D3000803230F4E0911C20F0E0E450F04E1082DC
:108D400060911C2070E0E0912120F09122208CEFB6
:108D50009FE1099510921C20FCCE1092482028CF4C
:108D60001F920F920FB60F9211240BB60F922F93F2
:108D70003F934F935F936F937F938F939F93AF93A3
:108D8000BF93EF93FF93E0912801F091290109959A
:108D9000E0911D20F0911E200995FF91EF91BF9168
:108DA000AF919F918F917F916F915F914F913F9183
:108DB0002F910F900BBE0F900FBE0F901F90189524
:108DC000E9E8F2E21382128288EE93E0A0E0B0E0DC
:108DD00084839583A683B7832CE631E03183208397
:108DE00025EC30E03587248724EC30E03787268770
:108DF00020EC30E0318B208B21EC30E0338B228B68
:108E000022EC30E0358B248B26EC30E0378B268B40
:108E1000118E128E138E148EE6E2F3E2138212820A
:108E200084839583A683B7832EE731E03183208343
:108E3000E2E3F3E220E520831182E4E3F3E215822A
:108E400016821186138642E050E060E070E04487AD
:108E500055876687778713A215A614A620E931E007
:108E600033A722A717A6EDE7F3E2138212828483C9
:108E70009583A683B7838CE991E091838083128EDA
:108E8000118E14860895789484B5836084BD85B569
:108E9000836085BD80916E00816080936E0082E06A
:108EA0008093810080918100816080938100809116
:108EB00080008160809380008091B1008460809305
:108EC000B1008091B00081608093B00080919100EA
:108ED00083608093910080919000816080939000E6
:108EE00087E880937A001092C10080E49AE10E94A2
:108EF00092499093702080936F20009709F458C096
:108F0000109271201092722090938520809384207B
:108F10008EE180937F2080EE80937E2010927720D8
:108F2000109278201092792010927A20109281204D
:108F30001092822088E49AE09093202080931F2052
:108F40000F9A559A17985D9A579A82EC80938000F1
:108F500089E1809381008CE280937B2087EC809371
:108F6000802087E08093832088E391E090937D20A8
:108F700080937C208FEF93E090938700809386000E
:108F80008AE490E0909389008093880089E391E0DF
:108F9000909376208093752083E29DE090931E202D
:108FA00080931D2081E080936F0078940E94D70603
:108FB0008CEF94E0909374208093732081E08093F1
:108FC0003420109226201092252010924C201092CE
:108FD0006E2010924A20809349201092422061E036
:108FE00081E10E94BA0861E080E10E94BA088091A4
:108FF000B9008E7F8093B9008091B9008D7F8093F6
:10900000B90088E48093B80085E48093BC008DE7C4
:1090100099E090932420809323208EE799E0909309
:109020002220809321208CE08093B80080912B2017
:10903000811188C061E082E00E94E808809163238A
:10904000882321F08EE593E20E94241810923F239A
:1090500010923D2310923A231092392382E080939C
:1090600038230E947109EB0161E0809138230E944E
:10907000E80861E0809138230E94BA081FB7F8948D
:1090800080912720811127C0E7E7F8E08491E7E984
:10909000F8E09491E82FF0E0EE0FFF1FE15AF74F50
:1090A000A591B491EC91E92321F461E084E00E9460
:1090B000BA0861E084E00E94E8088CB580618CBD4C
:1090C0008CB580648CBD61E087E00E94E80861E0B7
:1090D00085E00E94E808809127208F5F80932720F9
:1090E0001FBF82E580933223109233238091322375
:1090F000909133230E94AE0F1AE08FEF0E94890FE8
:109100001150D9F784E393E20E94B10F20E030E0E0
:10911000A90160E084E393E20E94C70F182F8093B7
:109120003E23813009F476C00E9471096C1B7D0BCF
:10913000613D774058F381E08093392384E393E2E3
:109140000E947E0FC8E160E08C2F0E94E80860E07A
:109150008C2F0E94BA08CF5FCE31A9F70E94241F3E
:1091600064E670E080E090E00E943E090E94D7062D
:1091700085ED94E00E946727C0903220D090332084
:109180008091302090913120C81AD90A0D2C000C02
:10919000EE08FF0881ED91E00E94FD2980E20E9427
:1091A0001B27C701B6010E94C0298AED91E00E94E9
:1091B000FD290E944A2780E180932C2086E080933D
:1091C0002F201092C00083E390E09093C50080931D
:1091D000C40088E18093C1008091C20080648093C4
:1091E000C2008091C20080628093C2008091C20060
:1091F00080618093C20010922E2010922D2084EE68
:109200009EE190932901809328010E94BA2C0E942C
:10921000A20EFBCF2AEA31E040E050E068E084E3B0
:1092200093E20E94C70F82FF2AC010933F238091D0
:109230003F23C12CD12C7601823029F4C12CD12CB2
:10924000E12C80E4F82E20E030E0A90167E384E31C
:1092500093E20E94C70FA701960169E284E393E2BB
:109260000E94C70F80933E238823C1F00E9471099A
:109270006C1B7D0B613D774030F388E05DCF14E0DF
:109280000E94900F80933E231150D1F78A3A11F03B
:1092900082E052CF82E080933F23C9CF80913F2369
:1092A0008230D1F420E030E0A9016AE384E393E264
:1092B0000E94C70F882311F086E03ECF0E94900FD6
:1092C000807C803C19F483E080933F230E94900FC0
:1092D0000E94900F0E94900F84E393E20E947E0F01
:1092E00080E5809332231092332381E00E94CD11D8
:1092F000882389F08EE593E20E949D14882309F467
:1093000021CF81E080932B2010922A2010922920D7
:109310001092282017CF80E00E94CD11882309F4F5
:1093200011CFE8CF0F931F93CF93DF938230910536
:1093300010F482E090E0E0919A23F0919B2330E0DA
:1093400020E0B0E0A0E0309799F42115310509F450
:109350004AC0281B390B24303105D8F58A819B81FE
:109360006115710589F1FB0193838283FE0111C0B0
:10937000408151810281138148175907E0F0481755
:10938000590799F4109761F012960C93129713965F
:109390001C933296CF01DF91CF911F910F910895C9
:1093A00000939A2310939B23F4CF2115310551F09C
:1093B0004217530738F0A901DB019A01BD01DF0113
:1093C000F801C1CFEF01F9CF90939B2380939A23AB
:1093D000CDCFFE01E20FF31F81939193225031090B
:1093E00039832883D7CF2091982330919923232B39
:1093F00041F420912C0130912D0130939923209339
:10940000982320912A0130912B012115310541F437
:109410002DB73EB740912E0150912F01241B350BE3
:10942000E0919823F0919923E217F307A0F42E1B03
:109430003F0B2817390778F0AC014E5F5F4F2417B8
:10944000350748F04E0F5F1F5093992340939823A0
:10945000819391939FCFF0E0E0E09CCFCF93DF9397
:109460000097E9F0FC01329713821282A0919A23AF
:10947000B0919B23ED0130E020E01097A1F4208112
:109480003181820F931F20919823309199232817BF
:10949000390709F061C0F0939923E0939823DF9195
:1094A000CF910895EA01CE17DF07E8F54A815B8185
:1094B0009E0141155105B1F7E901FB83EA8349910A
:1094C0005991C40FD51FEC17FD0761F4808191817C
:1094D0000296840F951FE901998388838281938185
:1094E0009B838A83F0E0E0E012968D919C91139724
:1094F0000097B9F52D913C911197CD010296820FFD
:10950000931F20919823309199232817390739F612
:10951000309751F510929B2310929A23B093992380
:10952000A0939823BCCFD383C28340815181840F01
:10953000951FC817D90761F44E5F5F4F88819981E5
:10954000480F591F518340838A819B819383828373
:109550002115310509F0B0CFF0939B23E0939A23B6
:109560009ECFFD01DC01C0CF13821282D7CF8F9234
:109570009F92AF92BF92CF92DF92EF92FF92CF93E2
:10958000DF93EC01688179818A819B816115710586
:109590008105910521F464E279ED8BE597E02DE1F9
:1095A00033EF41E050E00E94184E49015A019B01FF
:1095B000AC01A7EAB1E40E94374E6B017C01ACEE2E
:1095C000B4EFA50194010E94454EC60ED71EE81EB9
:1095D000F91EF7FE06C081E0C81AD108E10880E84C
:1095E000F80AC882D982EA82FB82C701B6019F7756
:1095F000DF91CF91FF90EF90DF90CF90BF90AF9031
:109600009F908F9008958F929F92AF92BF92CF922A
:10961000DF92EF92FF926091300170913101809161
:10962000320190913301611571058105910521F495
:1096300064E279ED8BE597E02DE133EF41E050E016
:109640000E94184E49015A019B01AC01A7EAB1E4FE
:109650000E94374E6B017C01ACEEB4EFA501940182
:109660000E94454EC60ED71EE81EF91EF7FE06C024
:1096700081E0C81AD108E10880E8F80AC0923001F8
:10968000D0923101E0923201F0923301C701B6016C
:109690009F77FF90EF90DF90CF90BF90AF909F901B
:1096A0008F9008956093300170933101809332015F
:1096B0009093330108952F923F924F925F926F9251
:1096C0007F928F929F92AF92BF92CF92DF92EF9252
:1096D000FF920F931F93CF93DF93CDB7DEB72B97F6
:1096E0000FB6F894DEBF0FBECDBF7C013B018A01EF
:1096F000FC0117821682838181FFDDC1CE010196B4
:109700005C01F7019381F30193FD859193FF8191B2
:109710003F01882309F453C1853239F493FD8591C3
:1097200093FF81913F01853229F4B70190E00E94B7
:10973000744DE7CF912C212C312CFFE1F31538F03B
:109740008B3211F190F4803209F1833229F137FC28
:109750003CC020ED280F2A3050F536FE20C08AE0AC
:10976000989E200D1124922E06C08D3291F08033E8
:1097700071F7689430F8F30193FD859193FF81911F
:109780003F018111DACF21C0689431F8689432F832
:10979000F2CF689433F8EFCF689434F8ECCFEAE076
:1097A0002E9E200D1124222E689435F8E4CF8E329F
:1097B00029F436FC04C1689436F8DDCF8C3619F4F0
:1097C000689437F8D8CF8836B1F2982F9F7D95549A
:1097D0009330E0F08336A1F18337C1F1833509F08E
:1097E00063C02801F2E04F0E511CF801C080D18007
:1097F000692D70E036FC02C06FEF7FEFC6010E945A
:109800005E4D4C01689437F882010AC00C5F1F4F0F
:10981000FFE3F98388248394912C6501E89437F859
:1098200033FE2DC0522C8114910471F5552009F49A
:1098300068CFB70180E290E00E94744D5A94F6CF51
:10984000F801808189830E5F1F4FE4CF2801F2E089
:109850004F0E511CF801C080D180692D70E036FC9C
:1098600002C06FEF7FEFC6010E94694D4C0182017B
:10987000D5CFB70180E290E00E94744D2A9428145D
:10988000190409F0B0F7CECFF60137FC859137FE09
:1098900081916F01B70190E00E94744D51105A946C
:1098A000F1E08F1A9108BFCF843619F0893609F09C
:1098B00077C0F80137FE6BC060817181828193812E
:1098C0000C5F1F4FF32DFF763F2E97FF09C0909539
:1098D0008095709561957F4F8F4F9F4F689437F8B3
:1098E0002AE030E0A5010E94A44DC82ECA188C2C95
:1098F000432C36FE0CC0E89440F8C91440F434FE02
:1099000005C032FC03C0F32DFE7E4F2E892C44FE91
:10991000AAC0FE01EC0DF11D8081803309F09CC0CE
:10992000242D297E422E842D8870582E43FCAAC0F7
:1099300040FEA4C09C2C821418F42C0C922C981875
:1099400044FEA6C0B70180E390E00E94744D42FE41
:1099500009C088E790E041FE02C088E590E0B701C9
:109960000E94744DC91408F49FC0CA94D12C9FEF73
:10997000C91AD90ACA0CDB1CF60182916F01B70122
:1099800090E00E94744DAC14BD04B1F74FCF6081DC
:109990007181072E000C880B990B0E5F1F4F92CF21
:1099A000D32CE894D4F82AE030E08537E1F1232D78
:1099B000297FD22E8F36A9F1F0F4883551F1F701C5
:1099C000868197812B960FB6F894DEBF0FBECDBF70
:1099D000DF91CF911F910F91FF90EF90DF90CF908B
:1099E000BF90AF909F908F907F906F905F904F90BF
:1099F0003F902F900895803749F0883701F7D4FEC3
:109A000002C06894D2F820E130E00DC06894D4F828
:109A1000F6CF34FE03C0822F8660D82E20E132E0DC
:109A200002C028E030E0F801D7FE0FC060817181EC
:109A3000828193810C5F1F4FA5010E94A44DC82E07
:109A4000CA183D2CE89437F852CF6081718190E0BC
:109A500080E00E5F1F4FF0CF42FC02C0839463CFC3
:109A60008394839460CF842D867809F45CCFF6CFFD
:109A7000B70180E290E00E94744D83948214C0F399
:109A8000512C5ECF522C5818821408F459CFF8CFBD
:109A9000842D867809F466CF8BE241FE80E247FC94
:109AA0008DE2B70190E05CCFB70180E390E00E94C7
:109AB000744D9A9457CF8FEF9FEF84CFFC010590A0
:109AC000615070400110D8F7809590958E0F9F1FC0
:109AD0000895FC016150704001900110D8F7809505
:109AE00090958E0F9F1F08950F931F93CF93DF9331
:109AF000182F092FEB018B8181FD09C01FEF0FEF9C
:109B0000812F902FDF91CF911F910F91089582FFA8
:109B100014C02E813F818C819D81281739073CF428
:109B2000E881F981CF0101969983888310838E8122
:109B30009F8101969F838E83E3CFE885F985812FEE
:109B40000995892BA1F3DACFFA01AA27283051F120
:109B5000203181F1E8946F936E7F6E5F7F4F8F4F5E
:109B60009F4FAF4FB1E03ED0B4E03CD0670F781FBD
:109B7000891F9A1FA11D680F791F8A1F911DA11DA2
:109B80006A0F711D811D911DA11D20D009F46894DB
:109B90003F912AE0269F11243019305D3193DEF683
:109BA000CF010895462F4770405D4193B3E00FD039
:109BB000C9F7F6CF462F4F70405D4A3318F0495D24
:109BC00031FD4052419302D0A9F7EACFB4E0A69507
:109BD0009795879577956795BA95C9F70097610529
:109BE000710508959B01AC010A2E0694579547957F
:109BF00037952795BA95C9F7620F731F841F951F74
:109C0000A01D0895F999FECF92BD81BDF89A9927BC
:109C100080B50895262FF999FECF1FBA92BD81BD58
:109C200020BD0FB6F894FA9AF99A0FBE01960895DE
:109C3000052E97FB1EF400940E942F4E57FD07D06F
:109C40000E944A4E07FC03D04EF40C942F4E5095C0
:109C50004095309521953F4F4F4F5F4F0895909518
:109C60008095709561957F4F8F4F9F4F08950E940B
:109C70006C4EA59F900DB49F900DA49F800D911DDB
:109C800011240895B7FF0C94374E0E94374E821B63
:109C9000930B0895A1E21A2EAA1BBB1BFD010DC058
:109CA000AA1FBB1FEE1FFF1FA217B307E407F5078C
:109CB00020F0A21BB30BE40BF50B661F771F881F68
:109CC000991F1A9469F760957095809590959B01FE
:109CD000AC01BD01CF010895A29FB001B39FC001A7
:109CE000A39F700D811D1124911DB29F700D811DC8
:109CF0001124911D08950E948F4E0C94774F0E945D
:109D0000704F58F00E94694F40F029F45F3F29F0EE
:109D10000C94604F51110C94AB4F0C94664F0E9401
:109D2000884F68F39923B1F3552391F3951B550B95
:109D3000BB27AA2762177307840738F09F5F5F4F1E
:109D4000220F331F441FAA1FA9F335D00E2E3AF05D
:109D5000E0E832D091505040E695001CCAF72BD075
:109D6000FE2F29D0660F771F881FBB1F26173707C6
:109D70004807AB07B0E809F0BB0B802DBF01FF27F8
:109D800093585F4F3AF09E3F510578F00C94604F26
:109D90000C94AB4F5F3FE4F3983ED4F386957795F0
:109DA0006795B795F7959F5FC9F7880F911D9695B1
:109DB000879597F90895E1E0660F771F881FBB1F0D
:109DC000621773078407BA0720F0621B730B840BBA
:109DD000BA0BEE1F88F7E09508950E94F44E689440
:109DE000B1110C94AB4F08950E94904F88F09F578B
:109DF00098F0B92F9927B751B0F0E1F0660F771FAF
:109E0000881F991F1AF0BA95C9F714C0B13091F0A4
:109E10000E94AA4FB1E008950C94AA4F672F782FA3
:109E20008827B85F39F0B93FCCF386957795679569
:109E3000B395D9F73EF490958095709561957F4FD5
:109E40008F4F9F4F0895E89409C097FB3EF490957B
:109E50008095709561957F4F8F4F9F4F9923A9F003
:109E6000F92F96E9BB279395F69587957795679592
:109E7000B795F111F8CFFAF4BB0F11F460FF1BC0D6
:109E80006F5F7F4F8F4F9F4F16C0882311F096E969
:109E900011C0772321F09EE8872F762F05C0662317
:109EA00071F096E8862F70E060E02AF09A95660FD0
:109EB000771F881FDAF7880F9695879597F9089589
:109EC00097F99F6780E870E060E008959FEF80EC6D
:109ED000089500240A941616170618060906089510
:109EE00000240A9412161306140605060895092E76
:109EF0000394000C11F4882352F0BB0F40F4BF2BE5
:109F000011F460FF04C06F5F7F4F8F4F9F4F089524
:109F100057FD9058440F551F59F05F3F71F047951A
:109F2000880F97FB991F61F09F3F79F087950895FF
:109F3000121613061406551FF2CF4695F1DF08C01E
:109F4000161617061806991FF1CF8695710561053B
:109F500008940895E894BB2766277727CB0197F9E3
:109F600008950E94C44F0C94774F0E94694F38F0B7
:109F70000E94704F20F0952311F00C94604F0C94C8
:109F8000664F11240C94AB4F0E94884F70F3959F3D
:109F9000C1F3950F50E0551F629FF001729FBB27E0
:109FA000F00DB11D639FAA27F00DB11DAA1F649F7C
:109FB0006627B00DA11D661F829F2227B00DA11D2F
:109FC000621F739FB00DA11D621F839FA00D611DB5
:109FD000221F749F3327A00D611D231F849F600DD6
:109FE000211D822F762F6A2F11249F5750409AF0FF
:109FF000F1F088234AF0EE0FFF1FBB1F661F771F8B
:10A00000881F91505040A9F79E3F510580F00C9455
:10A01000604F0C94AB4F5F3FE4F3983ED4F38695CA
:10A0200077956795B795F795E7959F5FC1F7FE2BF5
:10A03000880F911D9695879597F9089519F416F450
:10A040000C94664F0C9464500E94904FB8F399237F
:10A05000C9F3B6F39F57550B87FF0E947250002437
:10A06000A0E640EA900180585695979528F4805CC8
:10A07000660F771F881F20F026173707480730F430
:10A08000621B730B840B202931294A2BA695179448
:10A090000794202531254A2758F7660F771F881F18
:10A0A00020F026173707480730F4620B730B840B38
:10A0B000200D311D411DA09581F7B901842F9158C4
:10A0C000880F9695879508959F3F31F0915020F421
:10A0D000879577956795B795880F911D9695879584
:10A0E00097F9089591505040660F771F881FD2F757
:10A0F0000895AA1BBB1B51E107C0AA1FBB1FA617CF
:10A10000B70710F0A61BB70B881F991F5A95A9F720
:10A1100080959095BC01CD01089597FB072E16F40C
:10A12000009407D077FD09D00E94795007FC05D034
:10A130003EF4909581959F4F0895709561957F4F5E
:10A140000895EE0FFF1F0024001C0BBE0790F69130
:10A15000E02D0994FB01DC0104C08D910190801970
:10A1600021F441505040C8F7881B990B0895FB011A
:10A17000DC010D900020E9F7119701900D9200206D
:10A18000E1F70895FC018191861721F08823D9F722
:10A19000992708953197CF010895FB01DC018D9136
:10A1A000019080190110D9F3990B0895FB01DC018E
:10A1B00001900D920020E1F70895FB01DC01415070
:10A1C000504048F001900D920020C9F701C01D9247
:10A1D00041505040E0F70895FC0181E090E001908B
:10A1E000061609F4CF010020D1F7019708950F93C7
:10A1F0001F93CF93DF93CDB7DEB72E970FB6F894AA
:10A20000DEBF0FBECDBF0D891E8986E08C831A8309
:10A2100009838FEF9FE79E838D83AE01475E5F4F7B
:10A220006F89788DCE0101960E945B4B2F81388516
:10A23000020F131FF80110822E960FB6F894DEBF9E
:10A240000FBECDBFDF91CF911F910F910895F8946C
:02A25000FFCF3E
:10A252002F000000000000000000000000000000CD
:10A2620000000000000000000000000000000000EC
:10A27200FA00DF1AFFFFFFFF121C00009C23800080
:10A28200010000002F00000000000000000000009C
:10A29200000000000D0000000000000000000000AF
:10A2A20000000000000803000000007F0A00150BF8
:10A2B200000000001A00001900000000350E9F0D7A
:10A2C200CC0D820EFD0DDB0DEF0D00000000410FE5
:10A2D200140F750FEA0E0D0FFA0EEB0E00000000C0
:10A2E200491A9F0DC617AA1A00000000011BE41AA2
:10A2F200D41AAB1AB41A601B6A1B2F0030313233E6
:10A3020034353637383941424344454600204B42C2
:10A312002028002900206279746573002E4241537F
:10A322000031364B2052414D2000204241534943D7
:10A33200206279746573206672656500464F524DDE
:10A34200415454494E4720454550524F4D004445D3
:10A35200433A20004845583A2000464F524D415456
:10A3620054494E472049324320454550524F4D00F3
:10A37200204469726563746F7279206F6620433A74
:10A382000025732F2573005C002E2E00436172643A
:10A392003A20005344312E30005344322E300053C1
:10A3A20044484300556E6B6E6F776E00202020206C
:10A3B20020566F6C756D6520747970653A20464140
:10A3C2005400436C7573746572733A2000426C6F6B
:10A3D200636B73207820436C75737465723A200046
:10A3E200546F74616C20426C6F636B733A20005639
:10A3F2006F6C756D652073697A6520284B62293A06
:10A402002000566F6C756D652073697A6520284D42
:10A4120062293A200050726F6772616D206C6F6121
:10A422006465640042415349432052414D2073699F
:10A432007A6500737461636B206C696D6974005690
:10A4420061726961626C657300464F522F474F53C8
:10A45200554220737461636B00737031002E627316
:10A46200732073656374696F6E004672656520427E
:10A47200415349430046726565205352414D0042A3
:10A48200415349432053544152542020202020203C
:10A492002020200050524F4752414D20454E44202B
:10A4A2002020202020202020005641524941424CA9
:10A4B20045532020202020202020202020005354FB
:10A4C20041434B204C494D4954202020202020203C
:10A4D2002020005350312020202020202020202026
:10A4E20020202020202020002E42535320454E447D
:10A4F20020202020202020202020202000535241F4
:10A502004D20454E442020202020202020202020A5
:10A5120020334646466800546F74616C2073697A32
:10A522006500557365642073697A650046726565D6
:10A532002073697A650042415349432052414D3AA2
:10A5420020004D494E3A20004D41583A20004241E8
:10A552005349432052414D203D2000494E56414C23
:08A56200494420524547000066
:00000001FF
